 attach002aAgent00

 Timestamp is 54be7d68 (reproducible build file hash)

 Preferred load address is 0000000180000000

 Start         Length     Name                   Class
 0001:00000000 00003da0H .text$mn                CODE
 0001:00003da0 00000036H .text$mn$00             CODE
 0001:00003dd6 00000092H .text$x                 CODE
 0002:00000000 000001e8H .idata$5                DATA
 0002:000001e8 00000038H .00cfg                  DATA
 0002:00000220 00000008H .CRT$XCA                DATA
 0002:00000228 00000008H .CRT$XCZ                DATA
 0002:00000230 00000008H .CRT$XIA                DATA
 0002:00000238 00000008H .CRT$XIC                DATA
 0002:00000240 00000008H .CRT$XIZ                DATA
 0002:00000248 00000008H .CRT$XLA                DATA
 0002:00000250 00000008H .CRT$XLZ                DATA
 0002:00000258 00000008H .CRT$XPA                DATA
 0002:00000260 00000008H .CRT$XPZ                DATA
 0002:00000268 00000008H .CRT$XTA                DATA
 0002:00000270 00000010H .CRT$XTZ                DATA
 0002:00000278 00000000H .gehcont$y              DATA
 0002:00000278 00000000H .gfids$y                DATA
 0002:00000280 00002500H .rdata                  DATA
 0002:00002780 00000000H .rdata$CastGuardVftablesA DATA
 0002:00002780 00000000H .rdata$CastGuardVftablesC DATA
 0002:00002780 00000028H .rdata$T                DATA
 0002:000027a8 000000c0H .rdata$voltmd           DATA
 0002:00002868 00000320H .rdata$zzzdbg           DATA
 0002:00002b88 00000008H .rtc$IAA                DATA
 0002:00002b90 00000008H .rtc$IZZ                DATA
 0002:00002b98 00000008H .rtc$TAA                DATA
 0002:00002ba0 00000008H .rtc$TZZ                DATA
 0002:00002ba8 00000004H .tls                    DATA
 0002:00002bac 00000004H .tls$                   DATA
 0002:00002bb0 00000008H .tls$ZZZ                DATA
 0002:00002bb8 000003f8H .xdata                  DATA
 0002:00002fb0 00000354H .edata                  DATA
 0002:00003304 00000078H .idata$2                DATA
 0002:0000337c 00000014H .idata$3                DATA
 0002:00003390 000001e8H .idata$4                DATA
 0002:00003578 0000048eH .idata$6                DATA
 0003:00000000 000000a0H .data                   DATA
 0003:000000a0 0001b308H .bss                    DATA
 0004:00000000 00000438H .pdata                  DATA

  Address         Publics by Value              Rva+Base               Lib:Object

 0000:00000000       __AbsoluteZero             0000000000000000     <absolute>
 0000:00000000       ___safe_se_handler_count   0000000000000000     <absolute>
 0000:00000000       ___safe_se_handler_table   0000000000000000     <absolute>
 0000:00000000       __arm64x_extra_rfe_table   0000000000000000     <absolute>
 0000:00000000       __arm64x_extra_rfe_table_size 0000000000000000     <absolute>
 0000:00000000       __arm64x_native_entrypoint 0000000000000000     <absolute>
 0000:00000000       __arm64x_redirection_metadata 0000000000000000     <absolute>
 0000:00000000       __arm64x_redirection_metadata_count 0000000000000000     <absolute>
 0000:00000000       __dynamic_value_reloc_table 0000000000000000     <absolute>
 0000:00000000       __enclave_config           0000000000000000     <absolute>
 0000:00000000       __guard_check_icall_a64n_fptr 0000000000000000     <absolute>
 0000:00000000       __guard_eh_cont_count      0000000000000000     <absolute>
 0000:00000000       __guard_eh_cont_table      0000000000000000     <absolute>
 0000:00000000       __guard_fids_count         0000000000000000     <absolute>
 0000:00000000       __guard_fids_table         0000000000000000     <absolute>
 0000:00000000       __guard_iat_count          0000000000000000     <absolute>
 0000:00000000       __guard_iat_table          0000000000000000     <absolute>
 0000:00000000       __guard_longjmp_count      0000000000000000     <absolute>
 0000:00000000       __guard_longjmp_table      0000000000000000     <absolute>
 0000:00000000       __hybrid_auxiliary_iat     0000000000000000     <absolute>
 0000:00000000       __hybrid_auxiliary_iat_copy 0000000000000000     <absolute>
 0000:00000000       __hybrid_code_map          0000000000000000     <absolute>
 0000:00000000       __hybrid_code_map_count    0000000000000000     <absolute>
 0000:00000000       __x64_code_ranges_to_entry_points 0000000000000000     <absolute>
 0000:00000000       __x64_code_ranges_to_entry_points_count 0000000000000000     <absolute>
 0000:00000100       __guard_flags              0000000000000100     <absolute>
 0000:00000000       __ImageBase                0000000180000000     <linker-defined>
 0001:00000000       ?CallStaticVoidMethod@JNIEnv_@@QEAAXPEAV_jclass@@PEAU_jmethodID@@ZZ 0000000180001000 f i libattach002aAgent00.obj
 0001:00000024       ?NewObject@JNIEnv_@@QEAAPEAV_jobject@@PEAV_jclass@@PEAU_jmethodID@@ZZ 0000000180001024 f i libattach002aAgent00.obj
 0001:00000048       ?SetEventNotificationMode@_jvmtiEnv@@QEAA?AW4jvmtiError@@W4jvmtiEventMode@@W4jvmtiEvent@@PEAV_jobject@@ZZ 0000000180001048 f i libattach002aAgent00.obj
 0001:00000050       ?TranslateError@@YAPEBDW4jvmtiError@@@Z 0000000180001050 f   libattach002aAgent00.obj
 0001:00000308       ?nsk_jni_check_exception@@YAHPEAUJNIEnv_@@QEBDH@Z 0000000180001308 f   libattach002aAgent00.obj
 0001:0000044c       ?nsk_jni_lverify@@YAHHPEAUJNIEnv_@@HQEBDH1ZZ 000000018000144c f   libattach002aAgent00.obj
 0001:000004ec       Agent_OnAttach             00000001800014ec f   libattach002aAgent00.obj
 0001:000007c0       Java_nsk_jvmti_unit_FollowReferences_FollowRefObjects_addRefToVerify 00000001800017c0 f   libattach002aAgent00.obj
 0001:0000097c       Java_nsk_jvmti_unit_FollowReferences_FollowRefObjects_getTag 000000018000197c f   libattach002aAgent00.obj
 0001:00000a38       Java_nsk_jvmti_unit_FollowReferences_FollowRefObjects_resetRefsToVerify 0000000180001a38 f   libattach002aAgent00.obj
 0001:00000a40       Java_nsk_jvmti_unit_FollowReferences_FollowRefObjects_resetTags 0000000180001a40 f   libattach002aAgent00.obj
 0001:00000a84       Java_nsk_jvmti_unit_FollowReferences_FollowRefObjects_setTag 0000000180001a84 f   libattach002aAgent00.obj
 0001:00000cd0       Java_nsk_share_jvmti_ArgumentHandler_getAgentOptionsString 0000000180001cd0 f   libattach002aAgent00.obj
 0001:00000d7c       Java_nsk_share_jvmti_DebugeeClass_checkStatus 0000000180001d7c f   libattach002aAgent00.obj
 0001:00000e04       Java_nsk_share_jvmti_DebugeeClass_resetAgentData 0000000180001e04 f   libattach002aAgent00.obj
 0001:00000e64       Java_nsk_share_jvmti_RedefineAgent_agentStatus 0000000180001e64 f   libattach002aAgent00.obj
 0001:00000e70       Java_nsk_share_jvmti_RedefineAgent_isRedefined 0000000180001e70 f   libattach002aAgent00.obj
 0001:00000e7c       Java_nsk_share_jvmti_RedefineAgent_redefineAttempted 0000000180001e7c f   libattach002aAgent00.obj
 0001:00000e88       MA_checkStatus             0000000180001e88 f   libattach002aAgent00.obj
 0001:00000f2c       __local_stdio_printf_options 0000000180001f2c f i libattach002aAgent00.obj
 0001:00000f34       _snprintf                  0000000180001f34 f i libattach002aAgent00.obj
 0001:00001154       exitOnError                0000000180002154 f   libattach002aAgent00.obj
 0001:00001208       fprintf                    0000000180002208 f i libattach002aAgent00.obj
 0001:0000124c       nsk_aod_agentFinished      000000018000224c f   libattach002aAgent00.obj
 0001:0000143c       nsk_aod_agentLoaded        000000018000243c f   libattach002aAgent00.obj
 0001:0000167c       nsk_aod_createJNIEnv       000000018000267c f   libattach002aAgent00.obj
 0001:000016f4       nsk_aod_createOptions      00000001800026f4 f   libattach002aAgent00.obj
 0001:00001960       nsk_aod_getOptionValue     0000000180002960 f   libattach002aAgent00.obj
 0001:00001a4c       nsk_aod_internal_error     0000000180002a4c f   libattach002aAgent00.obj
 0001:00001a78       nsk_aod_optionSpecified    0000000180002a78 f   libattach002aAgent00.obj
 0001:00001b40       nsk_free_options           0000000180002b40 f   libattach002aAgent00.obj
 0001:00001ba0       nsk_jvmti_aod_deallocate   0000000180002ba0 f   libattach002aAgent00.obj
 0001:00001c54       nsk_jvmti_aod_disableEvents 0000000180002c54 f   libattach002aAgent00.obj
 0001:00001d24       nsk_jvmti_aod_disableEventsAndFinish 0000000180002d24 f   libattach002aAgent00.obj
 0001:00001d60       nsk_jvmti_aod_enableEvents 0000000180002d60 f   libattach002aAgent00.obj
 0001:00001e20       nsk_jvmti_aod_getClassName 0000000180002e20 f   libattach002aAgent00.obj
 0001:00001efc       nsk_jvmti_aod_redefineClass 0000000180002efc f   libattach002aAgent00.obj
 0001:00002174       nsk_jvmti_createJVMTIEnv   0000000180003174 f   libattach002aAgent00.obj
 0001:000022a4       nsk_jvmti_lverify          00000001800032a4 f   libattach002aAgent00.obj
 0001:00002394       nsk_jvmti_resetAgentData   0000000180003394 f   libattach002aAgent00.obj
 0001:00002408       nsk_lcomplain              0000000180003408 f   libattach002aAgent00.obj
 0001:00002428       nsk_ldisplay               0000000180003428 f   libattach002aAgent00.obj
 0001:00002448       nsk_ltrace                 0000000180003448 f   libattach002aAgent00.obj
 0001:00002468       nsk_lvcomplain             0000000180003468 f   libattach002aAgent00.obj
 0001:00002620       nsk_lvdisplay              0000000180003620 f   libattach002aAgent00.obj
 0001:0000266c       nsk_lverify                000000018000366c f   libattach002aAgent00.obj
 0001:000026c8       nsk_lvtrace                00000001800036c8 f   libattach002aAgent00.obj
 0001:00002728       nsk_printf                 0000000180003728 f   libattach002aAgent00.obj
 0001:00002750       nsk_vprintf                0000000180003750 f   libattach002aAgent00.obj
 0001:00002804       printf                     0000000180003804 f i libattach002aAgent00.obj
 0001:00002d04       vmObjectAllocHandler       0000000180003d04 f   libattach002aAgent00.obj
 0001:00002e6c       __raise_securityfailure    0000000180003e6c f   MSVCRT:gs_report.obj
 0001:00002ea0       __report_gsfailure         0000000180003ea0 f   MSVCRT:gs_report.obj
 0001:000030e0       __GSHandlerCheck           00000001800040e0 f   MSVCRT:gshandler.obj
 0001:00003100       __GSHandlerCheckCommon     0000000180004100 f   MSVCRT:gshandler.obj
 0001:00003170       __security_check_cookie    0000000180004170 f   MSVCRT:amdsecgs.obj
 0001:000034b0       _DllMainCRTStartup         00000001800044b0 f   MSVCRT:dll_dllmain.obj
 0001:000034f0       __scrt_acquire_startup_lock 00000001800044f0 f   MSVCRT:utility.obj
 0001:0000352c       __scrt_dllmain_after_initialize_c 000000018000452c f   MSVCRT:utility.obj
 0001:00003560       __scrt_dllmain_before_initialize_c 0000000180004560 f   MSVCRT:utility.obj
 0001:00003578       __scrt_dllmain_crt_thread_attach 0000000180004578 f   MSVCRT:utility.obj
 0001:000035a0       __scrt_dllmain_crt_thread_detach 00000001800045a0 f   MSVCRT:utility.obj
 0001:000035b8       __scrt_dllmain_exception_filter 00000001800045b8 f   MSVCRT:utility.obj
 0001:00003618       __scrt_dllmain_uninitialize_c 0000000180004618 f   MSVCRT:utility.obj
 0001:00003648       __scrt_dllmain_uninitialize_critical 0000000180004648 f   MSVCRT:utility.obj
 0001:0000365c       __scrt_initialize_crt      000000018000465c f   MSVCRT:utility.obj
 0001:000036a8       __scrt_initialize_onexit_tables 00000001800046a8 f   MSVCRT:utility.obj
 0001:00003734       __scrt_is_nonwritable_in_current_image 0000000180004734 f   MSVCRT:utility.obj
 0001:000037cc       __scrt_release_startup_lock 00000001800047cc f   MSVCRT:utility.obj
 0001:000037f0       __scrt_uninitialize_crt    00000001800047f0 f   MSVCRT:utility.obj
 0001:0000381c       _onexit                    000000018000481c f   MSVCRT:utility.obj
 0001:00003858       atexit                     0000000180004858 f   MSVCRT:utility.obj
 0001:00003870       __crt_debugger_hook        0000000180004870 f   MSVCRT:utility_desktop.obj
 0001:00003878       __scrt_fastfail            0000000180004878 f   MSVCRT:utility_desktop.obj
 0001:000039c4       _guard_check_icall_nop     00000001800049c4 f i MSVCRT:guard_support.obj
 0001:000039c8       __security_init_cookie     00000001800049c8 f   MSVCRT:gs_support.obj
 0001:00003a74       DllMain                    0000000180004a74 f   MSVCRT:dll_dllmain_stub.obj
 0001:00003a98       ?__scrt_initialize_type_info@@YAXXZ 0000000180004a98 f   MSVCRT:tncleanup.obj
 0001:00003aa8       ?__scrt_uninitialize_type_info@@YAXXZ 0000000180004aa8 f   MSVCRT:tncleanup.obj
 0001:00003ab4       __local_stdio_scanf_options 0000000180004ab4 f i MSVCRT:default_local_stdio_options.obj
 0001:00003abc       __scrt_initialize_default_local_stdio_options 0000000180004abc f   MSVCRT:default_local_stdio_options.obj
 0001:00003ad8       __scrt_get_dyn_tls_init_callback 0000000180004ad8 f   MSVCRT:dyn_tls_init.obj
 0001:00003ae0       _RTC_Initialize            0000000180004ae0 f   MSVCRT:initsect.obj
 0001:00003b1c       _RTC_Terminate             0000000180004b1c f   MSVCRT:initsect.obj
 0001:00003b58       __isa_available_init       0000000180004b58 f   MSVCRT:cpu_disp.obj
 0001:00003d04       _get_startup_argv_mode     0000000180004d04 f   MSVCRT:argv_mode.obj
 0001:00003d0c       __scrt_is_ucrt_dll_in_use  0000000180004d0c f   MSVCRT:ucrt_detection.obj
 0001:00003d20       memcpy                     0000000180004d20 f   vcruntime:VCRUNTIME140.dll
 0001:00003d26       memset                     0000000180004d26 f   vcruntime:VCRUNTIME140.dll
 0001:00003d2c       strchr                     0000000180004d2c f   vcruntime:VCRUNTIME140.dll
 0001:00003d32       __C_specific_handler       0000000180004d32 f   vcruntime:VCRUNTIME140.dll
 0001:00003d38       __std_type_info_destroy_list 0000000180004d38 f   vcruntime:VCRUNTIME140.dll
 0001:00003d3e       strcmp                     0000000180004d3e f   ucrt:api-ms-win-crt-string-l1-1-0.dll
 0001:00003d44       strcpy                     0000000180004d44 f   ucrt:api-ms-win-crt-string-l1-1-0.dll
 0001:00003d4a       strlen                     0000000180004d4a f   ucrt:api-ms-win-crt-string-l1-1-0.dll
 0001:00003d50       _initterm                  0000000180004d50 f   ucrt:api-ms-win-crt-runtime-l1-1-0.dll
 0001:00003d56       _initterm_e                0000000180004d56 f   ucrt:api-ms-win-crt-runtime-l1-1-0.dll
 0001:00003d5c       _seh_filter_dll            0000000180004d5c f   ucrt:api-ms-win-crt-runtime-l1-1-0.dll
 0001:00003d62       _configure_narrow_argv     0000000180004d62 f   ucrt:api-ms-win-crt-runtime-l1-1-0.dll
 0001:00003d68       _initialize_narrow_environment 0000000180004d68 f   ucrt:api-ms-win-crt-runtime-l1-1-0.dll
 0001:00003d6e       _initialize_onexit_table   0000000180004d6e f   ucrt:api-ms-win-crt-runtime-l1-1-0.dll
 0001:00003d74       _register_onexit_function  0000000180004d74 f   ucrt:api-ms-win-crt-runtime-l1-1-0.dll
 0001:00003d7a       _execute_onexit_table      0000000180004d7a f   ucrt:api-ms-win-crt-runtime-l1-1-0.dll
 0001:00003d80       _crt_atexit                0000000180004d80 f   ucrt:api-ms-win-crt-runtime-l1-1-0.dll
 0001:00003d86       _cexit                     0000000180004d86 f   ucrt:api-ms-win-crt-runtime-l1-1-0.dll
 0001:00003d8c       __acrt_initialize          0000000180004d8c f   MSVCRT:ucrt_stubs.obj
 0001:00003d8c       __acrt_thread_attach       0000000180004d8c f   MSVCRT:ucrt_stubs.obj
 0001:00003d8c       __acrt_thread_detach       0000000180004d8c f   MSVCRT:ucrt_stubs.obj
 0001:00003d8c       __acrt_uninitialize        0000000180004d8c f   MSVCRT:ucrt_stubs.obj
 0001:00003d8c       __acrt_uninitialize_critical 0000000180004d8c f   MSVCRT:ucrt_stubs.obj
 0001:00003d8c       __scrt_stub_for_acrt_initialize 0000000180004d8c f   MSVCRT:ucrt_stubs.obj
 0001:00003d8c       __scrt_stub_for_acrt_thread_attach 0000000180004d8c f   MSVCRT:ucrt_stubs.obj
 0001:00003d8c       __scrt_stub_for_acrt_thread_detach 0000000180004d8c f   MSVCRT:ucrt_stubs.obj
 0001:00003d8c       __scrt_stub_for_acrt_uninitialize 0000000180004d8c f   MSVCRT:ucrt_stubs.obj
 0001:00003d8c       __scrt_stub_for_acrt_uninitialize_critical 0000000180004d8c f   MSVCRT:ucrt_stubs.obj
 0001:00003d8c       __vcrt_initialize          0000000180004d8c f   MSVCRT:ucrt_stubs.obj
 0001:00003d8c       __vcrt_thread_attach       0000000180004d8c f   MSVCRT:ucrt_stubs.obj
 0001:00003d8c       __vcrt_thread_detach       0000000180004d8c f   MSVCRT:ucrt_stubs.obj
 0001:00003d8c       __vcrt_uninitialize        0000000180004d8c f   MSVCRT:ucrt_stubs.obj
 0001:00003d8c       __vcrt_uninitialize_critical 0000000180004d8c f   MSVCRT:ucrt_stubs.obj
 0001:00003d90       __scrt_stub_for_is_c_termination_complete 0000000180004d90 f   MSVCRT:ucrt_stubs.obj
 0001:00003d90       _is_c_termination_complete 0000000180004d90 f   MSVCRT:ucrt_stubs.obj
 0001:00003db0       _guard_dispatch_icall_nop  0000000180004db0 f   MSVCRT:guard_dispatch.obj
 0001:00003dd0       _guard_xfg_dispatch_icall_nop 0000000180004dd0 f   MSVCRT:guard_xfg_dispatch.obj
 0002:00000000       __imp_RtlCaptureContext    0000000180005000     kernel32:KERNEL32.dll
 0002:00000008       __imp_RtlLookupFunctionEntry 0000000180005008     kernel32:KERNEL32.dll
 0002:00000010       __imp_RtlVirtualUnwind     0000000180005010     kernel32:KERNEL32.dll
 0002:00000018       __imp_UnhandledExceptionFilter 0000000180005018     kernel32:KERNEL32.dll
 0002:00000020       __imp_SetUnhandledExceptionFilter 0000000180005020     kernel32:KERNEL32.dll
 0002:00000028       __imp_GetCurrentProcess    0000000180005028     kernel32:KERNEL32.dll
 0002:00000030       __imp_TerminateProcess     0000000180005030     kernel32:KERNEL32.dll
 0002:00000038       __imp_IsProcessorFeaturePresent 0000000180005038     kernel32:KERNEL32.dll
 0002:00000040       __imp_CloseHandle          0000000180005040     kernel32:KERNEL32.dll
 0002:00000048       __imp_InitializeCriticalSectionAndSpinCount 0000000180005048     kernel32:KERNEL32.dll
 0002:00000050       __imp_DeleteCriticalSection 0000000180005050     kernel32:KERNEL32.dll
 0002:00000058       __imp_CreateEventW         0000000180005058     kernel32:KERNEL32.dll
 0002:00000060       __imp_GetModuleHandleW     0000000180005060     kernel32:KERNEL32.dll
 0002:00000068       __imp_GetProcAddress       0000000180005068     kernel32:KERNEL32.dll
 0002:00000070       __imp_IsDebuggerPresent    0000000180005070     kernel32:KERNEL32.dll
 0002:00000078       __imp_QueryPerformanceCounter 0000000180005078     kernel32:KERNEL32.dll
 0002:00000080       __imp_GetCurrentProcessId  0000000180005080     kernel32:KERNEL32.dll
 0002:00000088       __imp_GetCurrentThreadId   0000000180005088     kernel32:KERNEL32.dll
 0002:00000090       __imp_GetSystemTimeAsFileTime 0000000180005090     kernel32:KERNEL32.dll
 0002:00000098       __imp_DisableThreadLibraryCalls 0000000180005098     kernel32:KERNEL32.dll
 0002:000000a0       __imp_InitializeSListHead  00000001800050a0     kernel32:KERNEL32.dll
 0002:000000a8       \177KERNEL32_NULL_THUNK_DATA 00000001800050a8     kernel32:KERNEL32.dll
 0002:000000b0       __imp_memcpy               00000001800050b0     vcruntime:VCRUNTIME140.dll
 0002:000000b8       __imp_memset               00000001800050b8     vcruntime:VCRUNTIME140.dll
 0002:000000c0       __imp_strchr               00000001800050c0     vcruntime:VCRUNTIME140.dll
 0002:000000c8       __imp___C_specific_handler 00000001800050c8     vcruntime:VCRUNTIME140.dll
 0002:000000d0       __imp___std_type_info_destroy_list 00000001800050d0     vcruntime:VCRUNTIME140.dll
 0002:000000d8       \177VCRUNTIME140_NULL_THUNK_DATA 00000001800050d8     vcruntime:VCRUNTIME140.dll
 0002:000000e0       __imp_malloc               00000001800050e0     ucrt:api-ms-win-crt-heap-l1-1-0.dll
 0002:000000e8       __imp_free                 00000001800050e8     ucrt:api-ms-win-crt-heap-l1-1-0.dll
 0002:000000f0       \177api-ms-win-crt-heap-l1-1-0_NULL_THUNK_DATA 00000001800050f0     ucrt:api-ms-win-crt-heap-l1-1-0.dll
 0002:000000f8       __imp__errno               00000001800050f8     ucrt:api-ms-win-crt-runtime-l1-1-0.dll
 0002:00000100       __imp_exit                 0000000180005100     ucrt:api-ms-win-crt-runtime-l1-1-0.dll
 0002:00000108       __imp__cexit               0000000180005108     ucrt:api-ms-win-crt-runtime-l1-1-0.dll
 0002:00000110       __imp__crt_atexit          0000000180005110     ucrt:api-ms-win-crt-runtime-l1-1-0.dll
 0002:00000118       __imp__execute_onexit_table 0000000180005118     ucrt:api-ms-win-crt-runtime-l1-1-0.dll
 0002:00000120       __imp__register_onexit_function 0000000180005120     ucrt:api-ms-win-crt-runtime-l1-1-0.dll
 0002:00000128       __imp__initialize_onexit_table 0000000180005128     ucrt:api-ms-win-crt-runtime-l1-1-0.dll
 0002:00000130       __imp__initialize_narrow_environment 0000000180005130     ucrt:api-ms-win-crt-runtime-l1-1-0.dll
 0002:00000138       __imp__configure_narrow_argv 0000000180005138     ucrt:api-ms-win-crt-runtime-l1-1-0.dll
 0002:00000140       __imp__seh_filter_dll      0000000180005140     ucrt:api-ms-win-crt-runtime-l1-1-0.dll
 0002:00000148       __imp__initterm_e          0000000180005148     ucrt:api-ms-win-crt-runtime-l1-1-0.dll
 0002:00000150       __imp__initterm            0000000180005150     ucrt:api-ms-win-crt-runtime-l1-1-0.dll
 0002:00000158       \177api-ms-win-crt-runtime-l1-1-0_NULL_THUNK_DATA 0000000180005158     ucrt:api-ms-win-crt-runtime-l1-1-0.dll
 0002:00000160       __imp___acrt_iob_func      0000000180005160     ucrt:api-ms-win-crt-stdio-l1-1-0.dll
 0002:00000168       __imp_ftell                0000000180005168     ucrt:api-ms-win-crt-stdio-l1-1-0.dll
 0002:00000170       __imp_fclose               0000000180005170     ucrt:api-ms-win-crt-stdio-l1-1-0.dll
 0002:00000178       __imp_fflush               0000000180005178     ucrt:api-ms-win-crt-stdio-l1-1-0.dll
 0002:00000180       __imp_fopen                0000000180005180     ucrt:api-ms-win-crt-stdio-l1-1-0.dll
 0002:00000188       __imp_fread                0000000180005188     ucrt:api-ms-win-crt-stdio-l1-1-0.dll
 0002:00000190       __imp_fseek                0000000180005190     ucrt:api-ms-win-crt-stdio-l1-1-0.dll
 0002:00000198       __imp___stdio_common_vsprintf 0000000180005198     ucrt:api-ms-win-crt-stdio-l1-1-0.dll
 0002:000001a0       __imp___stdio_common_vfprintf 00000001800051a0     ucrt:api-ms-win-crt-stdio-l1-1-0.dll
 0002:000001a8       __imp_rewind               00000001800051a8     ucrt:api-ms-win-crt-stdio-l1-1-0.dll
 0002:000001b0       \177api-ms-win-crt-stdio-l1-1-0_NULL_THUNK_DATA 00000001800051b0     ucrt:api-ms-win-crt-stdio-l1-1-0.dll
 0002:000001b8       __imp_strcmp               00000001800051b8     ucrt:api-ms-win-crt-string-l1-1-0.dll
 0002:000001c0       __imp_strcpy               00000001800051c0     ucrt:api-ms-win-crt-string-l1-1-0.dll
 0002:000001c8       __imp__strdup              00000001800051c8     ucrt:api-ms-win-crt-string-l1-1-0.dll
 0002:000001c8       __imp_strdup               00000001800051c8     ucrt:api-ms-win-crt-string-l1-1-0.dll
 0002:000001d0       __imp_strlen               00000001800051d0     ucrt:api-ms-win-crt-string-l1-1-0.dll
 0002:000001d8       __imp_strncpy              00000001800051d8     ucrt:api-ms-win-crt-string-l1-1-0.dll
 0002:000001e0       \177api-ms-win-crt-string-l1-1-0_NULL_THUNK_DATA 00000001800051e0     ucrt:api-ms-win-crt-string-l1-1-0.dll
 0002:000001e8       __guard_check_icall_fptr   00000001800051e8     MSVCRT:guard_support.obj
 0002:000001f0       __guard_xfg_check_icall_fptr 00000001800051f0     MSVCRT:guard_support.obj
 0002:000001f8       __guard_dispatch_icall_fptr 00000001800051f8     MSVCRT:guard_support.obj
 0002:00000200       __guard_xfg_dispatch_icall_fptr 0000000180005200     MSVCRT:guard_support.obj
 0002:00000208       __guard_xfg_table_dispatch_icall_fptr 0000000180005208     MSVCRT:guard_support.obj
 0002:00000210       __castguard_check_failure_os_handled_fptr 0000000180005210     MSVCRT:guard_support.obj
 0002:00000218       __guard_memcpy_fptr        0000000180005218     vcruntime:softmemtag.obj
 0002:00000220       __xc_a                     0000000180005220     MSVCRT:initializers.obj
 0002:00000228       __xc_z                     0000000180005228     MSVCRT:initializers.obj
 0002:00000230       __xi_a                     0000000180005230     MSVCRT:initializers.obj
 0002:00000240       __xi_z                     0000000180005240     MSVCRT:initializers.obj
 0002:00000248       __xl_a                     0000000180005248     MSVCRT:tlssup.obj
 0002:00000250       __xl_z                     0000000180005250     MSVCRT:tlssup.obj
 0002:00000258       __xp_a                     0000000180005258     MSVCRT:initializers.obj
 0002:00000260       __xp_z                     0000000180005260     MSVCRT:initializers.obj
 0002:00000268       __xt_a                     0000000180005268     MSVCRT:initializers.obj
 0002:00000270       __xt_z                     0000000180005270     MSVCRT:initializers.obj
 0002:00000280       ??_C@_0BG@IKDDPPGD@?$CILjava?1lang?1String?$DL?$CJV@ 0000000180005280     libattach002aAgent00.obj
 0002:000002a0       g_refKindStr               00000001800052a0     libattach002aAgent00.obj
 0002:00000450       ??_C@_09BPLDFGCI@unknown_0@ 0000000180005450     libattach002aAgent00.obj
 0002:00000460       ??_C@_0BL@FPNMECJD@JVMTI_HEAP_REFERENCE_CLASS@ 0000000180005460     libattach002aAgent00.obj
 0002:00000480       ??_C@_0BL@FKGKKLNM@JVMTI_HEAP_REFERENCE_FIELD@ 0000000180005480     libattach002aAgent00.obj
 0002:000004a0       ??_C@_0CD@CAEHCFJF@JVMTI_HEAP_REFERENCE_ARRAY_ELEM@ 00000001800054a0     libattach002aAgent00.obj
 0002:000004c8       ??_C@_0CC@DNEBMCNK@JVMTI_HEAP_REFERENCE_CLASS_LOAD@ 00000001800054c8     libattach002aAgent00.obj
 0002:000004f0       ??_C@_0BN@CJMIPEBB@JVMTI_HEAP_REFERENCE_SIGNERS@ 00000001800054f0     libattach002aAgent00.obj
 0002:00000510       ??_C@_0CH@HBOIDPEB@JVMTI_HEAP_REFERENCE_PROTECTION@ 0000000180005510     libattach002aAgent00.obj
 0002:00000538       ??_C@_0BP@MDKGDGKL@JVMTI_HEAP_REFERENCE_INTERFACE@ 0000000180005538     libattach002aAgent00.obj
 0002:00000558       ??_C@_0CC@JJMIHNJH@JVMTI_HEAP_REFERENCE_STATIC_FIE@ 0000000180005558     libattach002aAgent00.obj
 0002:00000580       ??_C@_0CD@IDHEEGID@JVMTI_HEAP_REFERENCE_CONSTANT_P@ 0000000180005580     libattach002aAgent00.obj
 0002:000005a8       ??_C@_0CA@EFFCHNG@JVMTI_HEAP_REFERENCE_SUPERCLASS@ 00000001800055a8     libattach002aAgent00.obj
 0002:000005c8       ??_C@_0L@PCDFHGCJ@unknown_11@ 00000001800055c8     libattach002aAgent00.obj
 0002:000005d8       ??_C@_0L@NJBICFOK@unknown_12@ 00000001800055d8     libattach002aAgent00.obj
 0002:000005e8       ??_C@_0L@MAADBEKL@unknown_13@ 00000001800055e8     libattach002aAgent00.obj
 0002:000005f8       ??_C@_0L@IPECICGM@unknown_14@ 00000001800055f8     libattach002aAgent00.obj
 0002:00000608       ??_C@_0L@JGFJLDCN@unknown_15@ 0000000180005608     libattach002aAgent00.obj
 0002:00000618       ??_C@_0L@LNHEOAOO@unknown_16@ 0000000180005618     libattach002aAgent00.obj
 0002:00000628       ??_C@_0L@KEGPNBKP@unknown_17@ 0000000180005628     libattach002aAgent00.obj
 0002:00000638       ??_C@_0L@CDPHMNGA@unknown_18@ 0000000180005638     libattach002aAgent00.obj
 0002:00000648       ??_C@_0L@DKOMPMCB@unknown_19@ 0000000180005648     libattach002aAgent00.obj
 0002:00000658       ??_C@_0L@OJGIPJDB@unknown_20@ 0000000180005658     libattach002aAgent00.obj
 0002:00000668       ??_C@_0CA@KAOFNDEM@JVMTI_HEAP_REFERENCE_JNI_GLOBAL@ 0000000180005668     libattach002aAgent00.obj
 0002:00000688       ??_C@_0CC@HPFAJBK@JVMTI_HEAP_REFERENCE_SYSTEM_CLA@ 0000000180005688     libattach002aAgent00.obj
 0002:000006b0       ??_C@_0BN@FDEGFOHC@JVMTI_HEAP_REFERENCE_MONITOR@ 00000001800056b0     libattach002aAgent00.obj
 0002:000006d0       ??_C@_0CB@HKIBCMAJ@JVMTI_HEAP_REFERENCE_STACK_LOCA@ 00000001800056d0     libattach002aAgent00.obj
 0002:000006f8       ??_C@_0BP@EAACMMOE@JVMTI_HEAP_REFERENCE_JNI_LOCAL@ 00000001800056f8     libattach002aAgent00.obj
 0002:00000718       ??_C@_0BM@IJDEOGOE@JVMTI_HEAP_REFERENCE_THREAD@ 0000000180005718     libattach002aAgent00.obj
 0002:00000738       ??_C@_0BL@EDGPPKC@JVMTI_HEAP_REFERENCE_OTHER@ 0000000180005738     libattach002aAgent00.obj
 0002:00000754       ??_C@_04BCJPDBDA@Code@     0000000180005754     libattach002aAgent00.obj
 0002:00000760       ??_C@_0BA@OCLMCFKC@LineNumberTable@ 0000000180005760     libattach002aAgent00.obj
 0002:00000770       ??_C@_0BD@CPAEPILC@LocalVariableTable@ 0000000180005770     libattach002aAgent00.obj
 0002:00000788       ??_C@_0BH@NMBDNHBD@LocalVariableTypeTable@ 0000000180005788     libattach002aAgent00.obj
 0002:000007a0       ??_C@_0O@HIHEEDNJ@StackMapTable@ 00000001800057a0     libattach002aAgent00.obj
 0002:000007b0       ??_C@_0CN@NKCKIIJI@nsk?1share?1aod?1TargetApplication@ 00000001800057b0     libattach002aAgent00.obj
 0002:000007e0       ??_C@_0M@OANFKLGH@agentLoaded@ 00000001800057e0     libattach002aAgent00.obj
 0002:000007f0       ??_C@_0O@JINEPNAJ@agentFinished@ 00000001800057f0     libattach002aAgent00.obj
 0002:00000800       ??_C@_0BH@BOPHNJNA@?$CILjava?1lang?1String?$DLZ?$CJV@ 0000000180005800     libattach002aAgent00.obj
 0002:00000818       ??_C@_0L@HCDIAMJG@?9?5?$CFs?0?5?$CFd?3?5@ 0000000180005818     libattach002aAgent00.obj
 0002:00000830       ??_C@_0JI@HLPECLFI@?$CD?5?4?4?4?6?$CD?5ERROR?3?5too?5many?5complai@ 0000000180005830     libattach002aAgent00.obj
 0002:000008d0       ??_C@_0ED@JNEKCCOB@The?5following?5fake?5exception?5st@ 00000001800058d0     libattach002aAgent00.obj
 0002:00000918       ??_C@_0CN@FCNMDFBH@nsk?4share?4Fake_Exception_for_RU@ 0000000180005918     libattach002aAgent00.obj
 0002:00000948       ??_C@_08PGFFNAEI@?$CI?$CFs?3?$CFd?$CJ?5@ 0000000180005948     libattach002aAgent00.obj
 0002:00000958       ??_C@_0DP@IENMAEGI@s?2test?2hotspot?2jtreg?2vmTestbase@ 0000000180005958     libattach002aAgent00.obj
 0002:00000998       ??_C@_0BL@NDJLFFJB@?7at?5nsk_lvcomplain?$CI?$CFs?3?$CFd?$CJ?6@ 0000000180005998     libattach002aAgent00.obj
 0002:000009b8       ??_C@_0BC@JOOKAFKF@?$CD?5ERROR?3?5?$CFs?0?5?$CFd?3?5@ 00000001800059b8     libattach002aAgent00.obj
 0002:000009d0       ??_C@_09KJEAHMEH@?$CD?5ERROR?3?5@ 00000001800059d0     libattach002aAgent00.obj
 0002:000009dc       ??_C@_02GPIOPFAK@?$DO?$DO@ 00000001800059dc     libattach002aAgent00.obj
 0002:000009e0       ??_C@_02FODMEDOG@?$DM?$DM@ 00000001800059e0     libattach002aAgent00.obj
 0002:000009e4       ??_C@_02DJGKEECL@?4?4@     00000001800059e4     libattach002aAgent00.obj
 0002:000009e8       ??_C@_0O@CJPGJOAF@?9?5?$CFs?0?5?$CFd?3?5?$CFs?5@ 00000001800059e8     libattach002aAgent00.obj
 0002:000009f8       ??_C@_0CB@IAKPDOIC@?$CD?5?5?5verified?5assertion?5is?5FALSE@ 00000001800059f8     libattach002aAgent00.obj
 0002:00000a20       ??_C@_0CO@LGONDEPD@stdout?3?5fflush?5failed?5?9?5err?$DN?$CFd?5@ 0000000180005a20     libattach002aAgent00.obj
 0002:00000a50       ??_C@_0CO@KBGKJPBD@stderr?3?5fflush?5failed?5?9?5err?$DN?$CFd?5@ 0000000180005a50     libattach002aAgent00.obj
 0002:00000a80       ??_C@_0BB@JCNMKLLK@JVMTI_ERROR_NONE@ 0000000180005a80     libattach002aAgent00.obj
 0002:00000a98       ??_C@_0BL@LDIMKLPH@JVMTI_ERROR_INVALID_THREAD@ 0000000180005a98     libattach002aAgent00.obj
 0002:00000ab8       ??_C@_0CB@PJFPAIKJ@JVMTI_ERROR_INVALID_THREAD_GROU@ 0000000180005ab8     libattach002aAgent00.obj
 0002:00000ae0       ??_C@_0BN@LLMKHMNF@JVMTI_ERROR_INVALID_PRIORITY@ 0000000180005ae0     libattach002aAgent00.obj
 0002:00000b00       ??_C@_0CB@MBOFKAGB@JVMTI_ERROR_THREAD_NOT_SUSPENDE@ 0000000180005b00     libattach002aAgent00.obj
 0002:00000b28       ??_C@_0BN@FABOLPBI@JVMTI_ERROR_THREAD_SUSPENDED@ 0000000180005b28     libattach002aAgent00.obj
 0002:00000b48       ??_C@_0BN@FDGNOBJM@JVMTI_ERROR_THREAD_NOT_ALIVE@ 0000000180005b48     libattach002aAgent00.obj
 0002:00000b68       ??_C@_0BL@GOBIFKNJ@JVMTI_ERROR_INVALID_OBJECT@ 0000000180005b68     libattach002aAgent00.obj
 0002:00000b88       ??_C@_0BK@FCMAJPPC@JVMTI_ERROR_INVALID_CLASS@ 0000000180005b88     libattach002aAgent00.obj
 0002:00000ba8       ??_C@_0BP@IKLLBKEB@JVMTI_ERROR_CLASS_NOT_PREPARED@ 0000000180005ba8     libattach002aAgent00.obj
 0002:00000bc8       ??_C@_0BN@KLPPLKG@JVMTI_ERROR_INVALID_METHODID@ 0000000180005bc8     libattach002aAgent00.obj
 0002:00000be8       ??_C@_0BN@BCEKOKND@JVMTI_ERROR_INVALID_LOCATION@ 0000000180005be8     libattach002aAgent00.obj
 0002:00000c08       ??_C@_0BM@DFDGPME@JVMTI_ERROR_INVALID_FIELDID@ 0000000180005c08     libattach002aAgent00.obj
 0002:00000c28       ??_C@_0BL@NELIEPEC@JVMTI_ERROR_NO_MORE_FRAMES@ 0000000180005c28     libattach002aAgent00.obj
 0002:00000c48       ??_C@_0BJ@BDBECFDM@JVMTI_ERROR_OPAQUE_FRAME@ 0000000180005c48     libattach002aAgent00.obj
 0002:00000c68       ??_C@_0BK@MIIFNLOB@JVMTI_ERROR_TYPE_MISMATCH@ 0000000180005c68     libattach002aAgent00.obj
 0002:00000c88       ??_C@_0BJ@HPCAOILC@JVMTI_ERROR_INVALID_SLOT@ 0000000180005c88     libattach002aAgent00.obj
 0002:00000ca8       ??_C@_0BG@CHILOPNI@JVMTI_ERROR_DUPLICATE@ 0000000180005ca8     libattach002aAgent00.obj
 0002:00000cc0       ??_C@_0BG@DIEMLHKM@JVMTI_ERROR_NOT_FOUND@ 0000000180005cc0     libattach002aAgent00.obj
 0002:00000cd8       ??_C@_0BM@NHMCKHOB@JVMTI_ERROR_INVALID_MONITOR@ 0000000180005cd8     libattach002aAgent00.obj
 0002:00000cf8       ??_C@_0BO@PPEDAJGL@JVMTI_ERROR_NOT_MONITOR_OWNER@ 0000000180005cf8     libattach002aAgent00.obj
 0002:00000d18       ??_C@_0BG@FCAIPEID@JVMTI_ERROR_INTERRUPT@ 0000000180005d18     libattach002aAgent00.obj
 0002:00000d30       ??_C@_0CB@EGDBNKOI@JVMTI_ERROR_INVALID_CLASS_FORMA@ 0000000180005d30     libattach002aAgent00.obj
 0002:00000d58       ??_C@_0CG@DGKOGIAL@JVMTI_ERROR_CIRCULAR_CLASS_DEFI@ 0000000180005d58     libattach002aAgent00.obj
 0002:00000d80       ??_C@_0BP@ICEALPKC@JVMTI_ERROR_FAILS_VERIFICATION@ 0000000180005d80     libattach002aAgent00.obj
 0002:00000da0       ??_C@_0DC@JDACLMIO@JVMTI_ERROR_UNSUPPORTED_REDEFIN@ 0000000180005da0     libattach002aAgent00.obj
 0002:00000dd8       ??_C@_0DE@GKDKNOMJ@JVMTI_ERROR_UNSUPPORTED_REDEFIN@ 0000000180005dd8     libattach002aAgent00.obj
 0002:00000e10       ??_C@_0BO@LAFKIOG@JVMTI_ERROR_INVALID_TYPESTATE@ 0000000180005e10     libattach002aAgent00.obj
 0002:00000e30       ??_C@_0DH@INDGCLLB@JVMTI_ERROR_UNSUPPORTED_REDEFIN@ 0000000180005e30     libattach002aAgent00.obj
 0002:00000e68       ??_C@_0DE@NHEOMMGI@JVMTI_ERROR_UNSUPPORTED_REDEFIN@ 0000000180005e68     libattach002aAgent00.obj
 0002:00000ea0       ??_C@_0CA@EKPNJOEP@JVMTI_ERROR_UNSUPPORTED_VERSION@ 0000000180005ea0     libattach002aAgent00.obj
 0002:00000ec0       ??_C@_0BN@OFFMAHHL@JVMTI_ERROR_NAMES_DONT_MATCH@ 0000000180005ec0     libattach002aAgent00.obj
 0002:00000ee0       ??_C@_0DN@HHBBLAKE@JVMTI_ERROR_UNSUPPORTED_REDEFIN@ 0000000180005ee0     libattach002aAgent00.obj
 0002:00000f20       ??_C@_0DO@HMBGBGNA@JVMTI_ERROR_UNSUPPORTED_REDEFIN@ 0000000180005f20     libattach002aAgent00.obj
 0002:00000f60       ??_C@_0BP@PBECGKHJ@JVMTI_ERROR_UNMODIFIABLE_CLASS@ 0000000180005f60     libattach002aAgent00.obj
 0002:00000f80       ??_C@_0BK@CANILEHF@JVMTI_ERROR_NOT_AVAILABLE@ 0000000180005f80     libattach002aAgent00.obj
 0002:00000fa0       ??_C@_0CE@INJKMEFK@JVMTI_ERROR_MUST_POSSESS_CAPABI@ 0000000180005fa0     libattach002aAgent00.obj
 0002:00000fc8       ??_C@_0BJ@LBFPFPDM@JVMTI_ERROR_NULL_POINTER@ 0000000180005fc8     libattach002aAgent00.obj
 0002:00000fe8       ??_C@_0BP@CHJPNNEM@JVMTI_ERROR_ABSENT_INFORMATION@ 0000000180005fe8     libattach002aAgent00.obj
 0002:00001008       ??_C@_0BP@OMFMNLC@JVMTI_ERROR_INVALID_EVENT_TYPE@ 0000000180006008     libattach002aAgent00.obj
 0002:00001028       ??_C@_0BN@BIBNPHHO@JVMTI_ERROR_ILLEGAL_ARGUMENT@ 0000000180006028     libattach002aAgent00.obj
 0002:00001048       ??_C@_0BK@KKNDHDCE@JVMTI_ERROR_NATIVE_METHOD@ 0000000180006048     libattach002aAgent00.obj
 0002:00001068       ??_C@_0BK@PMKCFHAE@JVMTI_ERROR_OUT_OF_MEMORY@ 0000000180006068     libattach002aAgent00.obj
 0002:00001088       ??_C@_0BK@NNJBDMNB@JVMTI_ERROR_ACCESS_DENIED@ 0000000180006088     libattach002aAgent00.obj
 0002:000010a8       ??_C@_0BI@GHECLMNC@JVMTI_ERROR_WRONG_PHASE@ 00000001800060a8     libattach002aAgent00.obj
 0002:000010c0       ??_C@_0BF@OLIHJOII@JVMTI_ERROR_INTERNAL@ 00000001800060c0     libattach002aAgent00.obj
 0002:000010d8       ??_C@_0BO@EOHGKJHI@JVMTI_ERROR_UNATTACHED_THREAD@ 00000001800060d8     libattach002aAgent00.obj
 0002:000010f8       ??_C@_0CA@LKHFDACL@JVMTI_ERROR_INVALID_ENVIRONMENT@ 00000001800060f8     libattach002aAgent00.obj
 0002:00001118       ??_C@_0BA@MMFHLOKK@?$DMunknown?5error?$DO@ 0000000180006118     libattach002aAgent00.obj
 0002:00001128       ??_C@_0CF@CBHOKDB@throwable?5?$DN?5jni?9?$DOExceptionOccur@ 0000000180006128     libattach002aAgent00.obj
 0002:00001150       ??_C@_03OFAPEBGM@?$CFs?6@  0000000180006150     libattach002aAgent00.obj
 0002:00001158       ??_C@_0DM@LPIGEGNJ@s?2test?2hotspot?2jtreg?2vmTestbase@ 0000000180006158     libattach002aAgent00.obj
 0002:00001198       ??_C@_0CC@NFCNPEPK@Exception?5in?5JNI?5call?5?$CIcleared?$CJ@ 0000000180006198     libattach002aAgent00.obj
 0002:000011c0       ??_C@_0BJ@IBAKFIKF@jni?9?$DOExceptionDescribe?$CI?$CJ@ 00000001800061c0     libattach002aAgent00.obj
 0002:000011e0       ??_C@_0BG@GGKALKMH@jni?9?$DOExceptionClear?$CI?$CJ@ 00000001800061e0     libattach002aAgent00.obj
 0002:000011f8       ??_C@_0CF@JMGFGJLJ@?$CD?5?5?5verified?5JNI?5assertion?5is?5F@ 00000001800061f8     libattach002aAgent00.obj
 0002:00001220       ??_C@_0CB@MLNJNCLJ@?5?5jvmti?5error?3?5code?$DN?$CFd?0?5name?$DN?$CFs@ 0000000180006220     libattach002aAgent00.obj
 0002:00001248       ??_C@_0CD@OHBGDKMK@?$CD?5?5?5jvmti?5error?3?5code?$DN?$CFd?0?5name?$DN@ 0000000180006248     libattach002aAgent00.obj
 0002:00001270       ??_C@_0CG@JNNCGPHB@?$CD?5?5?5error?5expected?3?5code?$DN?$CFd?0?5na@ 0000000180006270     libattach002aAgent00.obj
 0002:000012a0       ??_C@_0EB@IMGKPCGE@?$CIstr_obj?5?$DN?5jni?9?$DONewStringUTF?$CIco@ 00000001800062a0     libattach002aAgent00.obj
 0002:000012f0       ??_C@_0EA@HFOGGBCC@s?2test?2hotspot?2jtreg?2vmTestbase@ 00000001800062f0     libattach002aAgent00.obj
 0002:00001330       ??_C@_0M@KLIIGBGL@?$CFs?1?$CFs?4class@ 0000000180006330     libattach002aAgent00.obj
 0002:0000133c       ??_C@_02JDPG@rb@           000000018000633c     libattach002aAgent00.obj
 0002:00001340       ??_C@_0CF@OKNNGJPG@?$CD?5error?5occured?5while?5redefinin@ 0000000180006340     libattach002aAgent00.obj
 0002:00001368       ??_C@_05KKCIMGE@error@     0000000180006368     libattach002aAgent00.obj
 0002:00001370       ??_C@_0BD@HGNAOMCP@agent_data_monitor@ 0000000180006370     libattach002aAgent00.obj
 0002:00001390       ??_C@_0EB@OGCLGKLN@javaVM?9?$DOGetEnv?$CI?$CIvoid?5?$CK?$CK?$CJ?$CGjvmti_@ 0000000180006390     libattach002aAgent00.obj
 0002:000013e0       ??_C@_0EA@PNBCDMOA@s?2test?2hotspot?2jtreg?2vmTestbase@ 00000001800063e0     libattach002aAgent00.obj
 0002:00001420       ??_C@_0CI@DDPIFBGM@init_agent_data?$CIjvmti_env?0?5?$CGage@ 0000000180006420     libattach002aAgent00.obj
 0002:00001448       ??_C@_0DI@ILAHDLMP@?$CI?$CKagentThreadProc?$CJ?$CIjvmti_env?0?5a@ 0000000180006448     libattach002aAgent00.obj
 0002:00001480       ??_C@_0BD@KDBALNLB@JVMTI?5agent?5thread@ 0000000180006480     libattach002aAgent00.obj
 0002:00001498       ??_C@_0BB@NOKBFPFO@java?1lang?1Thread@ 0000000180006498     libattach002aAgent00.obj
 0002:000014ac       ??_C@_06FALKBLGB@?$DMinit?$DO@ 00000001800064ac     libattach002aAgent00.obj
 0002:000014c0       ??_C@_0EB@IFJBFEKC@?$CIthreadClass?5?$DN?5jni_env?9?$DOFindCla@ 00000001800064c0     libattach002aAgent00.obj
 0002:00001510       ??_C@_0GF@FGFIBKKL@?$CIthreadCtor?5?$DN?5jni_env?9?$DOGetMetho@ 0000000180006510     libattach002aAgent00.obj
 0002:00001578       ??_C@_0DN@NCPDJLOG@?$CIthreadName?5?$DN?5jni_env?9?$DONewStrin@ 0000000180006578     libattach002aAgent00.obj
 0002:000015c0       ??_C@_0FE@PFKODBGC@?$CIthreadObject?5?$DN?5jni_env?9?$DONewObj@ 00000001800065c0     libattach002aAgent00.obj
 0002:00001620       ??_C@_0ED@HOBAHHJI@?$CIthreadGlobalRef?5?$DN?5jni_env?9?$DONew@ 0000000180006620     libattach002aAgent00.obj
 0002:00001670       ??_C@_0FN@HNJJAHFC@jvmti_env?9?$DORunAgentThread?$CIagent@ 0000000180006670     libattach002aAgent00.obj
 0002:000016d0       ??_C@_0EA@MOJDNKDF@Debuggee?5status?5sync?5aborted?5be@ 00000001800066d0     libattach002aAgent00.obj
 0002:00001710       ??_C@_0EA@EEOEJAEN@status?5?$DN?5syncDebuggeeStatus?$CIjni@ 0000000180006710     libattach002aAgent00.obj
 0002:00001750       ??_C@_0BL@JBCFNBMB@nsk_jvmti_resetAgentData?$CI?$CJ@ 0000000180006750     libattach002aAgent00.obj
 0002:00001770       ??_C@_0EL@LPBEELIP@s?2test?2hotspot?2jtreg?2vmTestbase@ 0000000180006770     libattach002aAgent00.obj
 0002:000017c0       ??_C@_0CK@JDAMFDMJ@jvmti?9?$DOSetTag?$CIo?0?5tag?$CJ?5?$DN?$DN?5JVMTI_@ 00000001800067c0     libattach002aAgent00.obj
 0002:000017f0       ??_C@_0CC@DAMNHKNI@Can?8t?5set?5tag?5?$CFli?5for?5object?5?$CFl@ 00000001800067f0     libattach002aAgent00.obj
 0002:00001818       ??_C@_0DL@HAJPNKEF@jvmti?9?$DOGetObjectHashCode?$CIo?0?5?$CGha@ 0000000180006818     libattach002aAgent00.obj
 0002:00001858       ??_C@_0BL@JFPIEOBF@Can?8t?5get?5hash?5object?5?$CFlx?6@ 0000000180006858     libattach002aAgent00.obj
 0002:00001878       ??_C@_0BG@DICPHBKN@setTag?3?5?$CF08x?5?$DM?9?5?$CF?53li@ 0000000180006878     libattach002aAgent00.obj
 0002:00001890       ??_C@_0DH@FCEEBDMJ@?$CIs?5?$DN?5jni?9?$DOGetStringUTFChars?$CIsIn@ 0000000180006890     libattach002aAgent00.obj
 0002:000018c8       ??_C@_0BJ@OKKGHDCN@Can?8t?5get?5string?5at?5?$CF?$CDp?6@ 00000001800068c8     libattach002aAgent00.obj
 0002:000018e8       ??_C@_0BP@EKFLGGFJ@Can?8t?5get?5string?5at?5?$CF?$CDp?3?5null?6@ 00000001800068e8     libattach002aAgent00.obj
 0002:00001908       ??_C@_06ICODBHCL@?5?1?1?5?$CFs@ 0000000180006908     libattach002aAgent00.obj
 0002:00001910       ??_C@_0DB@KGFPLEGO@?$CIr?5?$DN?5jvmti?9?$DOGetTag?$CIo?0?5?$CGtag?$CJ?$CJ?5?$DN?$DN@ 0000000180006910     libattach002aAgent00.obj
 0002:00001948       ??_C@_0CO@PDAGBCGJ@Can?8t?5GetTag?5for?5object?5?$CFlx?4?5Re@ 0000000180006948     libattach002aAgent00.obj
 0002:00001978       ??_C@_0CH@HPEODOHC@TEST_BUG?3?5Max?4?5number?5of?5refs?5r@ 0000000180006978     libattach002aAgent00.obj
 0002:000019a0       ??_C@_0DI@PHFCABIM@?$CIr?5?$DN?5jvmti?9?$DOGetTag?$CIfrom?0?5?$CGtagFr@ 00000001800069a0     libattach002aAgent00.obj
 0002:000019d8       ??_C@_0DI@MDEGFNKD@TEST_BUG?3?5Can?8t?5GetTag?5for?5obje@ 00000001800069d8     libattach002aAgent00.obj
 0002:00001a10       ??_C@_0DE@MLELJAHM@?$CIr?5?$DN?5jvmti?9?$DOGetTag?$CIto?0?5?$CGtagTo?$CJ?$CJ@ 0000000180006a10     libattach002aAgent00.obj
 0002:00001a50       ??_C@_0EK@CABJMPML@WARNING?3?5some?5error?5happened?5in@ 0000000180006a50     libattach002aAgent00.obj
 0002:00001aa0       ??_C@_0DG@ECLJIGOO@s?2test?2hotspot?2jtreg?2vmTestbase@ 0000000180006aa0     libattach002aAgent00.obj
 0002:00001ad8       ??_C@_0CN@EDIMGGCE@options?5were?5not?5passed?5to?5the?5@ 0000000180006ad8     libattach002aAgent00.obj
 0002:00001b08       ??_C@_0BO@HIBNDEOE@Invalid?5options?5format?3?5?8?$CFs?8?6@ 0000000180006b08     libattach002aAgent00.obj
 0002:00001b28       ??_C@_0BG@BCGDCLLA@Option?5?8?$CFs?8?5is?5empty?6@ 0000000180006b28     libattach002aAgent00.obj
 0002:00001b40       ??_C@_0EI@CFFDGDKG@WARNING?3?5not?5all?5options?5were?5p@ 0000000180006b40     libattach002aAgent00.obj
 0002:00001b90       ??_C@_0EN@LHKBBCDP@?$CIoptions?5?$DN?5?$CIOptions?$CK?$CJ?5nsk_aod_c@ 0000000180006b90     libattach002aAgent00.obj
 0002:00001be0       ??_C@_0DM@MFFOLIAC@nsk_aod_optionSpecified?$CIoptions@ 0000000180006be0     libattach002aAgent00.obj
 0002:00001c20       ??_C@_0L@DALKGIIP@?9agentName@ 0000000180006c20     libattach002aAgent00.obj
 0002:00001c30       ??_C@_0BN@PFMBIOBG@Agent?5name?5wasn?8t?5specified?6@ 0000000180006c30     libattach002aAgent00.obj
 0002:00001c50       ??_C@_08FBJJFDKJ@?9verbose@ 0000000180006c50     libattach002aAgent00.obj
 0002:00001c5c       ??_C@_05LAPONLG@false@     0000000180006c5c     libattach002aAgent00.obj
 0002:00001c68       ??_C@_0BD@FMBAOLJK@options?5?$CB?$DN?5nullptr@ 0000000180006c68     libattach002aAgent00.obj
 0002:00001c80       ??_C@_0O@BPHJJCEJ@Options?5null?6@ 0000000180006c80     libattach002aAgent00.obj
 0002:00001c90       ??_C@_0BL@NJPPLGIO@Option?5?8?$CFs?8?5isn?8t?5defined?6@ 0000000180006c90     libattach002aAgent00.obj
 0002:00001cb0       ??_C@_0BE@DNNCOIDF@Agent?5?$CFs?5is?5loaded?6@ 0000000180006cb0     libattach002aAgent00.obj
 0002:00001cd0       ??_C@_0EJ@NDOPGKMK@?$CIlocalTargetAppClass?5?$DN?5jni?9?$DOFin@ 0000000180006cd0     libattach002aAgent00.obj
 0002:00001d20       ??_C@_0EO@HKMHFBAF@?$CItargetAppClass?5?$DN?5?$CIjclass?$CJ?5jni?9@ 0000000180006d20     libattach002aAgent00.obj
 0002:00001d70       ??_C@_0IB@FFOAAHNN@?$CIagentLoadedMethod?5?$DN?5jni?9?$DOGetSt@ 0000000180006d70     libattach002aAgent00.obj
 0002:00001df8       ??_C@_0DM@HLLJGLFL@?$CIagentNameString?5?$DN?5jni?9?$DONewStri@ 0000000180006df8     libattach002aAgent00.obj
 0002:00001e40       ??_C@_0FP@EEAOJLDE@?$CFs?3?5TEST?5LOGIC?5ERROR?3?5method?5?8a@ 0000000180006e40     libattach002aAgent00.obj
 0002:00001ea0       ??_C@_0II@KPBFKHFM@Status?5of?5agent?5?8?$CFs?8?5is?5?8passed@ 0000000180006ea0     libattach002aAgent00.obj
 0002:00001f28       ??_C@_0CB@ECJEOOED@Agent?5?$CFs?5finished?5?$CIsuccess?3?5?$CFd?$CJ@ 0000000180006f28     libattach002aAgent00.obj
 0002:00001f50       ??_C@_0IH@FIFEINGM@?$CIagentFinishedMethod?5?$DN?5jni?9?$DOGet@ 0000000180006f50     libattach002aAgent00.obj
 0002:00001fd8       ??_C@_0P@POOJKNDK@jni?5?$CB?$DN?5nullptr@ 0000000180006fd8     libattach002aAgent00.obj
 0002:00001ff0       ??_C@_0EC@LNOIGMCL@s?2test?2hotspot?2jtreg?2vmTestbase@ 0000000180006ff0     libattach002aAgent00.obj
 0002:00002038       ??_C@_0BH@DFACKHAD@jvmti?9?$DODeallocate?$CImem?$CJ@ 0000000180007038     libattach002aAgent00.obj
 0002:00002050       ??_C@_0BD@DPLLDHNC@Deallocate?5failed?6@ 0000000180007050     libattach002aAgent00.obj
 0002:00002068       ??_C@_0DF@HIDMGHGJ@jvmti?9?$DOGetClassSignature?$CIklass?0@ 0000000180007068     libattach002aAgent00.obj
 0002:000020a0       ??_C@_0BK@EEHGBOLL@Failed?5to?5get?5class?5name?6@ 00000001800070a0     libattach002aAgent00.obj
 0002:000020c0       ??_C@_0ED@MGJECIFJ@jvmti?9?$DOSetEventNotificationMode@ 00000001800070c0     libattach002aAgent00.obj
 0002:00002110       ??_C@_0EC@OOBBODLO@jvmti?9?$DOSetEventNotificationMode@ 0000000180007110     libattach002aAgent00.obj
 0002:00002158       ??_C@_0BD@FMNENHOF@?9pathToNewByteCode@ 0000000180007158     libattach002aAgent00.obj
 0002:00002170       ??_C@_0BN@ENCCFNI@Option?5?8?$CFs?8?5isn?8t?5specified?6@ 0000000180007170     libattach002aAgent00.obj
 0002:00002190       ??_C@_0BD@FPHHNGII@File?5name?5is?5null?6@ 0000000180007190     libattach002aAgent00.obj
 0002:000021a8       ??_C@_0BO@NOKNINPG@File?5with?5new?5bytecode?3?5?8?$CFs?8?6@ 00000001800071a8     libattach002aAgent00.obj
 0002:000021c8       ??_C@_0BJ@JMNBKGOB@Error?5opening?5file?5?8?$CFs?8?6@ 00000001800071c8     libattach002aAgent00.obj
 0002:000021e8       ??_C@_0BE@DFILLAPM@Opening?5file?5?8?$CFs?8?5?6@ 00000001800071e8     libattach002aAgent00.obj
 0002:00002200       ??_C@_0BA@EDGOILEI@File?5size?$DN?5?$CFld?6@ 0000000180007200     libattach002aAgent00.obj
 0002:00002210       ??_C@_0BM@OKBKDOLH@Failed?5to?5create?5memory?5?$CFs?6@ 0000000180007210     libattach002aAgent00.obj
 0002:00002230       ??_C@_0DF@NBFNDAJL@Failed?5to?5read?5all?5the?5bytes?0?5c@ 0000000180007230     libattach002aAgent00.obj
 0002:00002268       ??_C@_0BH@EINGAGAA@File?5read?5completely?5?6@ 0000000180007268     libattach002aAgent00.obj
 0002:00002280       ??_C@_0M@HJOJMJJL@Redefining?6@ 0000000180007280     libattach002aAgent00.obj
 0002:00002290       ??_C@_0DD@BFPGGFKG@?$CFs?3?5ObjectAlloc?5event?5received?5@ 0000000180007290     libattach002aAgent00.obj
 0002:000022d0       ??_C@_0FK@FBMCBLGK@s?2test?2hotspot?2jtreg?2vmTestbase@ 00000001800072d0     libattach002aAgent00.obj
 0002:00002330       ??_C@_0CB@BDIFGAGE@Ljava?1lang?1InterruptedException@ 0000000180007330     libattach002aAgent00.obj
 0002:00002360       ??_C@_0FF@IHMIMMEH@nsk_jvmti_aod_redefineClass?$CIopt@ 0000000180007360     libattach002aAgent00.obj
 0002:000023b8       ??_C@_0BP@MPALLHPL@java?1lang?1InterruptedException@ 00000001800073b8     libattach002aAgent00.obj
 0002:000023d8       ??_C@_0BO@ICIIEIIA@?$CFs?3?5failed?5to?5redefine?5class?6@ 00000001800073d8     libattach002aAgent00.obj
 0002:000023f8       ??_C@_0BB@CGPOECH@jvmti?5?$CB?$DN?5nullptr@ 00000001800073f8     libattach002aAgent00.obj
 0002:00002410       ??_C@_0BO@DBKDIPGD@jvmti?9?$DOAddCapabilities?$CI?$CGcaps?$CJ@ 0000000180007410     libattach002aAgent00.obj
 0002:00002430       ??_C@_0EC@ODFGFOAJ@jvmti?9?$DOSetEventCallbacks?$CI?$CGevent@ 0000000180007430     libattach002aAgent00.obj
 0002:00002478       ??_C@_0BN@GGABIMJA@?$CFs?3?5initialization?5was?5done?6@ 0000000180007478     libattach002aAgent00.obj
 0002:00002498       ??_C@_0CE@PACICCLF@nsk_aod_agentLoaded?$CIjni?0?5agentN@ 0000000180007498     libattach002aAgent00.obj
 0002:000024d0       ??_C@_1EC@JIJBPKFM@?$AAa?$AAp?$AAi?$AA?9?$AAm?$AAs?$AA?9?$AAw?$AAi?$AAn?$AA?9?$AAc?$AAo?$AAr?$AAe@ 00000001800074d0     MSVCRT:thread_safe_statics.obj
 0002:00002518       ??_C@_1BK@MGMFAEKH@?$AAk?$AAe?$AAr?$AAn?$AAe?$AAl?$AA3?$AA2?$AA?4?$AAd?$AAl?$AAl@ 0000000180007518     MSVCRT:thread_safe_statics.obj
 0002:00002538       ??_C@_0BJ@JEBJOJFJ@SleepConditionVariableCS@ 0000000180007538     MSVCRT:thread_safe_statics.obj
 0002:00002558       ??_C@_0BJ@PGPPEPCC@WakeAllConditionVariable@ 0000000180007558     MSVCRT:thread_safe_statics.obj
 0002:00002578       _pDefaultRawDllMain        0000000180007578     MSVCRT:dll_dllmain.obj
 0002:00002578       _pRawDllMain               0000000180007578     MSVCRT:dll_dllmain.obj
 0002:00002580       __xmm@ffffffffffffffffffffffffffffffff 0000000180007580     MSVCRT:utility.obj
 0002:00002590       _load_config_used          0000000180007590     MSVCRT:loadcfg.obj
 0002:00002780       _tls_used                  0000000180007780     MSVCRT:tlssup.obj
 0002:000027a8       __volatile_metadata        00000001800077a8     <linker-defined>
 0002:00002b88       __rtc_iaa                  0000000180007b88     MSVCRT:initsect.obj
 0002:00002b90       __rtc_izz                  0000000180007b90     MSVCRT:initsect.obj
 0002:00002b98       __rtc_taa                  0000000180007b98     MSVCRT:initsect.obj
 0002:00002ba0       __rtc_tzz                  0000000180007ba0     MSVCRT:initsect.obj
 0002:00002ba8       _tls_start                 0000000180007ba8     MSVCRT:tlssup.obj
 0002:00002bac       _Init_thread_epoch         0000000180007bac     MSVCRT:thread_safe_statics.obj
 0002:00002bb0       _tls_end                   0000000180007bb0     MSVCRT:tlssup.obj
 0002:00003304       __IMPORT_DESCRIPTOR_KERNEL32 0000000180008304     kernel32:KERNEL32.dll
 0002:00003318       __IMPORT_DESCRIPTOR_VCRUNTIME140 0000000180008318     vcruntime:VCRUNTIME140.dll
 0002:0000332c       __IMPORT_DESCRIPTOR_api-ms-win-crt-heap-l1-1-0 000000018000832c     ucrt:api-ms-win-crt-heap-l1-1-0.dll
 0002:00003340       __IMPORT_DESCRIPTOR_api-ms-win-crt-runtime-l1-1-0 0000000180008340     ucrt:api-ms-win-crt-runtime-l1-1-0.dll
 0002:00003354       __IMPORT_DESCRIPTOR_api-ms-win-crt-stdio-l1-1-0 0000000180008354     ucrt:api-ms-win-crt-stdio-l1-1-0.dll
 0002:00003368       __IMPORT_DESCRIPTOR_api-ms-win-crt-string-l1-1-0 0000000180008368     ucrt:api-ms-win-crt-string-l1-1-0.dll
 0002:0000337c       __NULL_IMPORT_DESCRIPTOR   000000018000837c     kernel32:KERNEL32.dll
 0003:0000005c       _Init_global_epoch         000000018000905c     MSVCRT:thread_safe_statics.obj
 0003:00000060       __security_cookie          0000000180009060     MSVCRT:gs_cookie.obj
 0003:00000068       __security_cookie_complement 0000000180009068     MSVCRT:gs_cookie.obj
 0003:00000070       __scrt_native_dllmain_reason 0000000180009070     MSVCRT:utility.obj
 0003:00000078       __isa_available            0000000180009078     MSVCRT:cpu_disp.obj
 0003:0000007c       __isa_enabled              000000018000907c     MSVCRT:cpu_disp.obj
 0003:00000080       __memset_fast_string_threshold 0000000180009080     MSVCRT:cpu_disp.obj
 0003:00000088       __memset_nt_threshold      0000000180009088     MSVCRT:cpu_disp.obj
 0003:00000090       __scrt_ucrt_dll_is_in_use  0000000180009090     MSVCRT:ucrt_stubs.obj
 0003:000000a0       g_wrongHeapCallbacks       00000001800090a0     libattach002aAgent00.obj
 0003:00000120       g_szTagInfo                0000000180009120     libattach002aAgent00.obj
 0003:00002060       g_tagFlags                 000000018000b060     libattach002aAgent00.obj
 0003:00002448       g_refsToVerifyCnt          000000018000b448     libattach002aAgent00.obj
 0003:0000244c       g_fakeUserData             000000018000b44c     libattach002aAgent00.obj
 0003:00002450       g_tagVisitCount            000000018000b450     libattach002aAgent00.obj
 0003:000033f0       g_refsToVerify             000000018000c3f0     libattach002aAgent00.obj
 0003:0001aaf0       g_userDataError            0000000180023af0     libattach002aAgent00.obj
 0003:0001ab00       multiagentsOptions         0000000180023b00     libattach002aAgent00.obj
 0003:0001ad60       ?_OptionsStorage@?1??__local_stdio_printf_options@@9@4_KA 0000000180023d60     libattach002aAgent00.obj
 0003:0001b328       _tls_index                 0000000180024328     MSVCRT:tlssup.obj
 0003:0001b330       __scrt_current_native_startup_state 0000000180024330     MSVCRT:utility.obj
 0003:0001b338       __scrt_native_startup_lock 0000000180024338     MSVCRT:utility.obj
 0003:0001b378       __scrt_debugger_hook_flag  0000000180024378     MSVCRT:utility_desktop.obj
 0003:0001b380       ?__type_info_root_node@@3U__type_info_node@@A 0000000180024380     MSVCRT:tncleanup.obj
 0003:0001b390       ?_OptionsStorage@?1??__local_stdio_scanf_options@@9@4_KA 0000000180024390     MSVCRT:default_local_stdio_options.obj
 0003:0001b398       __favor                    0000000180024398     MSVCRT:cpu_disp.obj
 0003:0001b3a0       __dyn_tls_init_callback    00000001800243a0     <common>

 entry point at        0001:000034b0

 Static symbols

 0000:fffd9000       .debug$S                   0000000180000000     attach002aAgent00.exp
 0000:fffd9000       .debug$S                   0000000180000000     vcruntime:VCRUNTIME140.dll
 0000:fffd9000       .debug$S                   0000000180000000     vcruntime:VCRUNTIME140.dll
 0000:fffd9000       .debug$S                   0000000180000000     vcruntime:VCRUNTIME140.dll
 0000:fffd9000       .debug$S                   0000000180000000     vcruntime:VCRUNTIME140.dll
 0000:fffd9000       .debug$S                   0000000180000000     vcruntime:VCRUNTIME140.dll
 0000:fffd9000       .debug$S                   0000000180000000     vcruntime:VCRUNTIME140.dll
 0000:fffd9000       .debug$S                   0000000180000000     vcruntime:VCRUNTIME140.dll
 0000:fffd9000       .debug$S                   0000000180000000     ucrt:api-ms-win-crt-convert-l1-1-0.dll
 0002:ffffb000       .idata$6                   0000000180000000     ucrt:api-ms-win-crt-convert-l1-1-0.dll
 0000:fffd9000       .debug$S                   0000000180000000     ucrt:api-ms-win-crt-heap-l1-1-0.dll
 0000:fffd9000       .debug$S                   0000000180000000     ucrt:api-ms-win-crt-heap-l1-1-0.dll
 0000:fffd9000       .debug$S                   0000000180000000     ucrt:api-ms-win-crt-heap-l1-1-0.dll
 0000:fffd9000       .debug$S                   0000000180000000     ucrt:api-ms-win-crt-heap-l1-1-0.dll
 0000:fffd9000       .debug$S                   0000000180000000     ucrt:api-ms-win-crt-runtime-l1-1-0.dll
 0000:fffd9000       .debug$S                   0000000180000000     ucrt:api-ms-win-crt-runtime-l1-1-0.dll
 0000:fffd9000       .debug$S                   0000000180000000     ucrt:api-ms-win-crt-runtime-l1-1-0.dll
 0000:fffd9000       .debug$S                   0000000180000000     ucrt:api-ms-win-crt-runtime-l1-1-0.dll
 0000:fffd9000       .debug$S                   0000000180000000     ucrt:api-ms-win-crt-runtime-l1-1-0.dll
 0000:fffd9000       .debug$S                   0000000180000000     ucrt:api-ms-win-crt-runtime-l1-1-0.dll
 0000:fffd9000       .debug$S                   0000000180000000     ucrt:api-ms-win-crt-runtime-l1-1-0.dll
 0000:fffd9000       .debug$S                   0000000180000000     ucrt:api-ms-win-crt-runtime-l1-1-0.dll
 0000:fffd9000       .debug$S                   0000000180000000     ucrt:api-ms-win-crt-runtime-l1-1-0.dll
 0000:fffd9000       .debug$S                   0000000180000000     ucrt:api-ms-win-crt-runtime-l1-1-0.dll
 0000:fffd9000       .debug$S                   0000000180000000     ucrt:api-ms-win-crt-runtime-l1-1-0.dll
 0000:fffd9000       .debug$S                   0000000180000000     ucrt:api-ms-win-crt-runtime-l1-1-0.dll
 0000:fffd9000       .debug$S                   0000000180000000     ucrt:api-ms-win-crt-runtime-l1-1-0.dll
 0000:fffd9000       .debug$S                   0000000180000000     ucrt:api-ms-win-crt-runtime-l1-1-0.dll
 0000:fffd9000       .debug$S                   0000000180000000     ucrt:api-ms-win-crt-runtime-l1-1-0.dll
 0000:fffd9000       .debug$S                   0000000180000000     ucrt:api-ms-win-crt-runtime-l1-1-0.dll
 0000:fffd9000       .debug$S                   0000000180000000     ucrt:api-ms-win-crt-stdio-l1-1-0.dll
 0000:fffd9000       .debug$S                   0000000180000000     ucrt:api-ms-win-crt-stdio-l1-1-0.dll
 0000:fffd9000       .debug$S                   0000000180000000     ucrt:api-ms-win-crt-stdio-l1-1-0.dll
 0000:fffd9000       .debug$S                   0000000180000000     ucrt:api-ms-win-crt-stdio-l1-1-0.dll
 0000:fffd9000       .debug$S                   0000000180000000     ucrt:api-ms-win-crt-stdio-l1-1-0.dll
 0000:fffd9000       .debug$S                   0000000180000000     ucrt:api-ms-win-crt-stdio-l1-1-0.dll
 0000:fffd9000       .debug$S                   0000000180000000     ucrt:api-ms-win-crt-stdio-l1-1-0.dll
 0000:fffd9000       .debug$S                   0000000180000000     ucrt:api-ms-win-crt-stdio-l1-1-0.dll
 0000:fffd9000       .debug$S                   0000000180000000     ucrt:api-ms-win-crt-stdio-l1-1-0.dll
 0000:fffd9000       .debug$S                   0000000180000000     ucrt:api-ms-win-crt-stdio-l1-1-0.dll
 0000:fffd9000       .debug$S                   0000000180000000     ucrt:api-ms-win-crt-string-l1-1-0.dll
 0000:fffd9000       .debug$S                   0000000180000000     ucrt:api-ms-win-crt-string-l1-1-0.dll
 0000:fffd9000       .debug$S                   0000000180000000     ucrt:api-ms-win-crt-string-l1-1-0.dll
 0000:fffd9000       .debug$S                   0000000180000000     ucrt:api-ms-win-crt-string-l1-1-0.dll
 0000:fffd9000       .debug$S                   0000000180000000     ucrt:api-ms-win-crt-string-l1-1-0.dll
 0000:fffd9000       .debug$S                   0000000180000000     ucrt:api-ms-win-crt-string-l1-1-0.dll
 0000:fffd9000       .debug$S                   0000000180000000     ucrt:api-ms-win-crt-string-l1-1-0.dll
 0000:fffd9000       .debug$S                   0000000180000000     ucrt:api-ms-win-crt-string-l1-1-0.dll
 0000:fffd9000       .debug$S                   0000000180000000     ucrt:api-ms-win-crt-string-l1-1-0.dll
 0000:fffd9000       .debug$S                   0000000180000000     kernel32:KERNEL32.dll
 0000:fffd9000       .debug$S                   0000000180000000     kernel32:KERNEL32.dll
 0000:fffd9000       .debug$S                   0000000180000000     kernel32:KERNEL32.dll
 0000:fffd9000       .debug$S                   0000000180000000     kernel32:KERNEL32.dll
 0000:fffd9000       .debug$S                   0000000180000000     kernel32:KERNEL32.dll
 0000:fffd9000       .debug$S                   0000000180000000     kernel32:KERNEL32.dll
 0000:fffd9000       .debug$S                   0000000180000000     kernel32:KERNEL32.dll
 0000:fffd9000       .debug$S                   0000000180000000     kernel32:KERNEL32.dll
 0000:fffd9000       .debug$S                   0000000180000000     kernel32:KERNEL32.dll
 0000:fffd9000       .debug$S                   0000000180000000     kernel32:KERNEL32.dll
 0000:fffd9000       .debug$S                   0000000180000000     kernel32:KERNEL32.dll
 0000:fffd9000       .debug$S                   0000000180000000     kernel32:KERNEL32.dll
 0000:fffd9000       .debug$S                   0000000180000000     kernel32:KERNEL32.dll
 0000:fffd9000       .debug$S                   0000000180000000     kernel32:KERNEL32.dll
 0000:fffd9000       .debug$S                   0000000180000000     kernel32:KERNEL32.dll
 0000:fffd9000       .debug$S                   0000000180000000     kernel32:KERNEL32.dll
 0000:fffd9000       .debug$S                   0000000180000000     kernel32:KERNEL32.dll
 0000:fffd9000       .debug$S                   0000000180000000     kernel32:KERNEL32.dll
 0000:fffd9000       .debug$S                   0000000180000000     kernel32:KERNEL32.dll
 0000:fffd9000       .debug$S                   0000000180000000     kernel32:KERNEL32.dll
 0000:fffd9000       .debug$S                   0000000180000000     kernel32:KERNEL32.dll
 0000:fffd9000       .debug$S                   0000000180000000     kernel32:KERNEL32.dll
 0000:fffd9000       .debug$S                   0000000180000000     kernel32:KERNEL32.dll
 0000:fffd9000       .debug$S                   0000000180000000     kernel32:KERNEL32.dll
 0000:fffd9000       .debug$S                   0000000180000000     kernel32:KERNEL32.dll
 0000:fffd9000       .debug$S                   0000000180000000     kernel32:KERNEL32.dll
 0000:fffd9000       .debug$S                   0000000180000000     kernel32:KERNEL32.dll
 0000:fffd9000       .debug$S                   0000000180000000     kernel32:KERNEL32.dll
 0001:00000f8c       addRefToVerify             0000000180001f8c f   libattach002aAgent00.obj
 0001:00001000       agentThreadWrapper         0000000180002000 f   libattach002aAgent00.obj
 0001:000011d8       file_basename              00000001800021d8 f   libattach002aAgent00.obj
 0001:00002858       startAgentThreadWrapper    0000000180003858 f   libattach002aAgent00.obj
 0001:00002b84       syncDebuggeeStatus         0000000180003b84 f   libattach002aAgent00.obj
 0001:00002f74       capture_previous_context   0000000180003f74 f   MSVCRT:gs_report.obj
 0001:00002fe8       ?__scrt_initialize_thread_safe_statics@@YAHXZ 0000000180003fe8 f   MSVCRT:thread_safe_statics.obj
 0001:000030b8       ?__scrt_uninitialize_thread_safe_statics@@YAXXZ 00000001800040b8 f   MSVCRT:thread_safe_statics.obj
 0001:00003160       $$000000                   0000000180004160     MSVCRT:amdsecgs.obj
 0001:00003190       ?dllmain_crt_dispatch@@YAHQEAUHINSTANCE__@@KQEAX@Z 0000000180004190 f   MSVCRT:dll_dllmain.obj
 0001:000031e0       ?dllmain_crt_process_attach@@YAHQEAUHINSTANCE__@@QEAX@Z 00000001800041e0 f   MSVCRT:dll_dllmain.obj
 0001:000032f8       ?dllmain_crt_process_detach@@YAH_N@Z 00000001800042f8 f   MSVCRT:dll_dllmain.obj
 0001:0000337c       ?dllmain_dispatch@@YAHQEAUHINSTANCE__@@KQEAX@Z 000000018000437c f   MSVCRT:dll_dllmain.obj
 0001:00003da0       $$000000                   0000000180004da0     MSVCRT:guard_dispatch.obj
 0001:00003dc0       $$000000                   0000000180004dc0     MSVCRT:guard_xfg_dispatch.obj
 0001:00003dd6       ?fin$0@?0??dllmain_crt_process_attach@@YAHQEAUHINSTANCE__@@QEAX@Z@4HA 0000000180004dd6 f   MSVCRT:dll_dllmain.obj
 0001:00003ded       ?fin$0@?0??dllmain_crt_process_detach@@YAH_N@Z@4HA 0000000180004ded f   MSVCRT:dll_dllmain.obj
 0001:00003e06       ?fin$1@?0??dllmain_crt_process_detach@@YAH_N@Z@4HA 0000000180004e06 f   MSVCRT:dll_dllmain.obj
 0001:00003e1a       ?filt$0@?0??dllmain_dispatch@@YAHQEAUHINSTANCE__@@KQEAX@Z@4HA 0000000180004e1a f   MSVCRT:dll_dllmain.obj
 0001:00003e50       __scrt_is_nonwritable_in_current_image$filt$0 0000000180004e50 f   MSVCRT:utility.obj
 0002:00000238       ?__scrt_initialize_tss_var@@3P6AHXZEA 0000000180005238     MSVCRT:thread_safe_statics.obj
 0002:00000380       ?opcLengths@@3QBEB         0000000180005380     libattach002aAgent00.obj
 0002:000024c0       GS_ExceptionPointers       00000001800074c0     MSVCRT:gs_report.obj
 0002:00002bb8       $unwind$fprintf            0000000180007bb8     libattach002aAgent00.obj
 0002:00002bc4       $unwind$printf             0000000180007bc4     libattach002aAgent00.obj
 0002:00002bd0       $unwind$_snprintf          0000000180007bd0     libattach002aAgent00.obj
 0002:00002be0       $unwind$?CallStaticVoidMethod@JNIEnv_@@QEAAXPEAV_jclass@@PEAU_jmethodID@@ZZ 0000000180007be0     libattach002aAgent00.obj
 0002:00002be0       $unwind$?NewObject@JNIEnv_@@QEAAPEAV_jobject@@PEAV_jclass@@PEAU_jmethodID@@ZZ 0000000180007be0     libattach002aAgent00.obj
 0002:00002be0       $unwind$nsk_lcomplain      0000000180007be0     libattach002aAgent00.obj
 0002:00002be0       $unwind$nsk_ldisplay       0000000180007be0     libattach002aAgent00.obj
 0002:00002be8       $unwind$nsk_jvmti_aod_disableEventsAndFinish 0000000180007be8     libattach002aAgent00.obj
 0002:00002be8       $unwind$nsk_lvdisplay      0000000180007be8     libattach002aAgent00.obj
 0002:00002be8       $unwind$_RTC_Initialize    0000000180007be8     MSVCRT:initsect.obj
 0002:00002be8       $unwind$_RTC_Terminate     0000000180007be8     MSVCRT:initsect.obj
 0002:00002be8       $unwind$?__scrt_initialize_thread_safe_statics@@YAHXZ 0000000180007be8     MSVCRT:thread_safe_statics.obj
 0002:00002bf4       $unwind$nsk_lvcomplain     0000000180007bf4     libattach002aAgent00.obj
 0002:00002c0c       $unwind$nsk_ltrace         0000000180007c0c     libattach002aAgent00.obj
 0002:00002c0c       $unwind$__report_gsfailure 0000000180007c0c     MSVCRT:gs_report.obj
 0002:00002c14       $unwind$nsk_lvtrace        0000000180007c14     libattach002aAgent00.obj
 0002:00002c14       $unwind$__raise_securityfailure 0000000180007c14     MSVCRT:gs_report.obj
 0002:00002c14       $unwind$__scrt_initialize_crt 0000000180007c14     MSVCRT:utility.obj
 0002:00002c14       $unwind$__scrt_initialize_onexit_tables 0000000180007c14     MSVCRT:utility.obj
 0002:00002c14       $unwind$__scrt_release_startup_lock 0000000180007c14     MSVCRT:utility.obj
 0002:00002c14       $unwind$__scrt_uninitialize_crt 0000000180007c14     MSVCRT:utility.obj
 0002:00002c14       $unwind$_onexit            0000000180007c14     MSVCRT:utility.obj
 0002:00002c1c       $unwind$nsk_lverify        0000000180007c1c     libattach002aAgent00.obj
 0002:00002c2c       $unwind$nsk_vprintf        0000000180007c2c     libattach002aAgent00.obj
 0002:00002c3c       $unwind$nsk_printf         0000000180007c3c     libattach002aAgent00.obj
 0002:00002c44       $unwind$Agent_OnAttach     0000000180007c44     libattach002aAgent00.obj
 0002:00002c68       $unwind$?nsk_jni_lverify@@YAHHPEAUJNIEnv_@@HQEBDH1ZZ 0000000180007c68     libattach002aAgent00.obj
 0002:00002c7c       $unwind$?nsk_jni_check_exception@@YAHPEAUJNIEnv_@@QEBDH@Z 0000000180007c7c     libattach002aAgent00.obj
 0002:00002c98       $unwind$nsk_jvmti_createJVMTIEnv 0000000180007c98     libattach002aAgent00.obj
 0002:00002cac       $unwind$Java_nsk_jvmti_unit_FollowReferences_FollowRefObjects_resetTags 0000000180007cac     libattach002aAgent00.obj
 0002:00002cac       $unwind$addRefToVerify     0000000180007cac     libattach002aAgent00.obj
 0002:00002cac       $unwind$nsk_aod_internal_error 0000000180007cac     libattach002aAgent00.obj
 0002:00002cac       $unwind$nsk_jvmti_resetAgentData 0000000180007cac     libattach002aAgent00.obj
 0002:00002cac       $unwind$__scrt_initialize_default_local_stdio_options 0000000180007cac     MSVCRT:default_local_stdio_options.obj
 0002:00002cac       $unwind$?dllmain_crt_dispatch@@YAHQEAUHINSTANCE__@@KQEAX@Z 0000000180007cac     MSVCRT:dll_dllmain.obj
 0002:00002cac       $unwind$DllMain            0000000180007cac     MSVCRT:dll_dllmain_stub.obj
 0002:00002cac       $unwind$__GSHandlerCheck   0000000180007cac     MSVCRT:gshandler.obj
 0002:00002cac       $unwind$?__scrt_uninitialize_thread_safe_statics@@YAXXZ 0000000180007cac     MSVCRT:thread_safe_statics.obj
 0002:00002cac       $unwind$__scrt_acquire_startup_lock 0000000180007cac     MSVCRT:utility.obj
 0002:00002cac       $unwind$__scrt_dllmain_after_initialize_c 0000000180007cac     MSVCRT:utility.obj
 0002:00002cac       $unwind$__scrt_dllmain_before_initialize_c 0000000180007cac     MSVCRT:utility.obj
 0002:00002cac       $unwind$__scrt_dllmain_crt_thread_attach 0000000180007cac     MSVCRT:utility.obj
 0002:00002cac       $unwind$__scrt_dllmain_crt_thread_detach 0000000180007cac     MSVCRT:utility.obj
 0002:00002cac       $unwind$__scrt_dllmain_uninitialize_c 0000000180007cac     MSVCRT:utility.obj
 0002:00002cac       $unwind$__scrt_dllmain_uninitialize_critical 0000000180007cac     MSVCRT:utility.obj
 0002:00002cac       $unwind$atexit             0000000180007cac     MSVCRT:utility.obj
 0002:00002cb4       $unwind$nsk_jvmti_lverify  0000000180007cb4     libattach002aAgent00.obj
 0002:00002cc8       $unwind$exitOnError        0000000180007cc8     libattach002aAgent00.obj
 0002:00002cd8       $unwind$Java_nsk_share_jvmti_ArgumentHandler_getAgentOptionsString 0000000180007cd8     libattach002aAgent00.obj
 0002:00002cd8       $unwind$nsk_jvmti_aod_deallocate 0000000180007cd8     libattach002aAgent00.obj
 0002:00002cec       $unwind$Java_nsk_jvmti_unit_FollowReferences_FollowRefObjects_getTag 0000000180007cec     libattach002aAgent00.obj
 0002:00002cec       $unwind$Java_nsk_share_jvmti_DebugeeClass_checkStatus 0000000180007cec     libattach002aAgent00.obj
 0002:00002cec       $unwind$agentThreadWrapper 0000000180007cec     libattach002aAgent00.obj
 0002:00002cfc       $unwind$nsk_aod_agentLoaded 0000000180007cfc     libattach002aAgent00.obj
 0002:00002cfc       $unwind$startAgentThreadWrapper 0000000180007cfc     libattach002aAgent00.obj
 0002:00002d18       $unwind$syncDebuggeeStatus 0000000180007d18     libattach002aAgent00.obj
 0002:00002d18       $unwind$__scrt_dllmain_exception_filter 0000000180007d18     MSVCRT:utility.obj
 0002:00002d2c       $unwind$Java_nsk_share_jvmti_DebugeeClass_resetAgentData 0000000180007d2c     libattach002aAgent00.obj
 0002:00002d2c       $unwind$nsk_aod_createJNIEnv 0000000180007d2c     libattach002aAgent00.obj
 0002:00002d34       $unwind$MA_checkStatus     0000000180007d34     libattach002aAgent00.obj
 0002:00002d48       $unwind$Java_nsk_jvmti_unit_FollowReferences_FollowRefObjects_setTag 0000000180007d48     libattach002aAgent00.obj
 0002:00002d60       $unwind$Java_nsk_jvmti_unit_FollowReferences_FollowRefObjects_addRefToVerify 0000000180007d60     libattach002aAgent00.obj
 0002:00002d7c       $unwind$nsk_aod_createOptions 0000000180007d7c     libattach002aAgent00.obj
 0002:00002d98       $unwind$nsk_aod_getOptionValue 0000000180007d98     libattach002aAgent00.obj
 0002:00002d98       $unwind$nsk_aod_optionSpecified 0000000180007d98     libattach002aAgent00.obj
 0002:00002dac       $unwind$nsk_aod_agentFinished 0000000180007dac     libattach002aAgent00.obj
 0002:00002dc8       $unwind$nsk_free_options   0000000180007dc8     libattach002aAgent00.obj
 0002:00002dd8       $unwind$nsk_jvmti_aod_getClassName 0000000180007dd8     libattach002aAgent00.obj
 0002:00002dec       $unwind$nsk_jvmti_aod_enableEvents 0000000180007dec     libattach002aAgent00.obj
 0002:00002e04       $unwind$nsk_jvmti_aod_disableEvents 0000000180007e04     libattach002aAgent00.obj
 0002:00002e1c       $unwind$nsk_jvmti_aod_redefineClass 0000000180007e1c     libattach002aAgent00.obj
 0002:00002e3c       $unwind$vmObjectAllocHandler 0000000180007e3c     libattach002aAgent00.obj
 0002:00002e5c       $unwind$capture_previous_context 0000000180007e5c     MSVCRT:gs_report.obj
 0002:00002e68       $unwind$__GSHandlerCheckCommon 0000000180007e68     MSVCRT:gshandler.obj
 0002:00002e70       $xdatasym                  0000000180007e70     MSVCRT:amdsecgs.obj
 0002:00002e74       $unwind$?dllmain_crt_process_attach@@YAHQEAUHINSTANCE__@@QEAX@Z 0000000180007e74     MSVCRT:dll_dllmain.obj
 0002:00002eb0       $unwind$?fin$0@?0??dllmain_crt_process_attach@@YAHQEAUHINSTANCE__@@QEAX@Z@4HA 0000000180007eb0     MSVCRT:dll_dllmain.obj
 0002:00002eb0       $unwind$?fin$0@?0??dllmain_crt_process_detach@@YAH_N@Z@4HA 0000000180007eb0     MSVCRT:dll_dllmain.obj
 0002:00002eb0       $unwind$?fin$1@?0??dllmain_crt_process_detach@@YAH_N@Z@4HA 0000000180007eb0     MSVCRT:dll_dllmain.obj
 0002:00002eb8       $unwind$?dllmain_crt_process_detach@@YAH_N@Z 0000000180007eb8     MSVCRT:dll_dllmain.obj
 0002:00002f0c       $unwind$?dllmain_dispatch@@YAHQEAUHINSTANCE__@@KQEAX@Z 0000000180007f0c     MSVCRT:dll_dllmain.obj
 0002:00002f34       $unwind$?filt$0@?0??dllmain_dispatch@@YAHQEAUHINSTANCE__@@KQEAX@Z@4HA 0000000180007f34     MSVCRT:dll_dllmain.obj
 0002:00002f3c       $unwind$_DllMainCRTStartup 0000000180007f3c     MSVCRT:dll_dllmain.obj
 0002:00002f4c       $unwind$__scrt_is_nonwritable_in_current_image 0000000180007f4c     MSVCRT:utility.obj
 0002:00002f6c       $unwind$__scrt_is_nonwritable_in_current_image$filt$0 0000000180007f6c     MSVCRT:utility.obj
 0002:00002f74       $unwind$__scrt_fastfail    0000000180007f74     MSVCRT:utility_desktop.obj
 0002:00002f84       $unwind$__security_init_cookie 0000000180007f84     MSVCRT:gs_support.obj
 0002:00002f90       $unwind$__isa_available_init 0000000180007f90     MSVCRT:cpu_disp.obj
 0002:00002fa0       $xdatasym                  0000000180007fa0     MSVCRT:guard_dispatch.obj
 0002:00002fa8       $xdatasym                  0000000180007fa8     MSVCRT:guard_xfg_dispatch.obj
 0002:00002fb0       .edata                     0000000180007fb0     attach002aAgent00.exp
 0002:00002fd8       rgpv                       0000000180007fd8     attach002aAgent00.exp
 0002:0000300c       rgszName                   000000018000800c     attach002aAgent00.exp
 0002:00003040       rgwOrd                     0000000180008040     attach002aAgent00.exp
 0002:0000305a       szName                     000000018000805a     attach002aAgent00.exp
 0002:00003070       $N00001                    0000000180008070     attach002aAgent00.exp
 0002:0000307f       $N00002                    000000018000807f     attach002aAgent00.exp
 0002:000030c4       $N00003                    00000001800080c4     attach002aAgent00.exp
 0002:00003101       $N00004                    0000000180008101     attach002aAgent00.exp
 0002:00003149       $N00005                    0000000180008149     attach002aAgent00.exp
 0002:00003189       $N00006                    0000000180008189     attach002aAgent00.exp
 0002:000031c6       $N00007                    00000001800081c6     attach002aAgent00.exp
 0002:00003201       $N00008                    0000000180008201     attach002aAgent00.exp
 0002:0000322f       $N00009                    000000018000822f     attach002aAgent00.exp
 0002:00003260       $N00010                    0000000180008260     attach002aAgent00.exp
 0002:0000328f       $N00011                    000000018000828f     attach002aAgent00.exp
 0002:000032be       $N00012                    00000001800082be     attach002aAgent00.exp
 0002:000032f3       $N00013                    00000001800082f3     attach002aAgent00.exp
 0002:00003762       .idata$6                   0000000180008762     kernel32:KERNEL32.dll
 0002:000037c6       .idata$6                   00000001800087c6     vcruntime:VCRUNTIME140.dll
 0002:00003982       .idata$6                   0000000180008982     ucrt:api-ms-win-crt-heap-l1-1-0.dll
 0002:000039a2       .idata$6                   00000001800089a2     ucrt:api-ms-win-crt-runtime-l1-1-0.dll
 0002:000039c4       .idata$6                   00000001800089c4     ucrt:api-ms-win-crt-stdio-l1-1-0.dll
 0002:000039e4       .idata$6                   00000001800089e4     ucrt:api-ms-win-crt-string-l1-1-0.dll
 0003:00000000       ?codeAttributeName@@3PEBDEB 0000000180009000     libattach002aAgent00.obj
 0003:00000008       ?lineNumberAttributeName@@3PEBDEB 0000000180009008     libattach002aAgent00.obj
 0003:00000010       ?localVarAttributeName@@3PEBDEB 0000000180009010     libattach002aAgent00.obj
 0003:00000018       ?localVarTypeAttributeName@@3PEBDEB 0000000180009018     libattach002aAgent00.obj
 0003:00000020       ?stackMapAttributeName@@3PEBDEB 0000000180009020     libattach002aAgent00.obj
 0003:00000028       ?callBytes@@3PAEA          0000000180009028     libattach002aAgent00.obj
 0003:0000002c       ?allocBytes@@3PAEA         000000018000902c     libattach002aAgent00.obj
 0003:00000030       TARGET_APP_CLASS_NAME      0000000180009030     libattach002aAgent00.obj
 0003:00000038       AGENT_LOADED_METHOD_NAME   0000000180009038     libattach002aAgent00.obj
 0003:00000040       AGENT_LOADED_METHOD_SIGNATURE 0000000180009040     libattach002aAgent00.obj
 0003:00000048       AGENT_FINISHED_METHOD_NAME 0000000180009048     libattach002aAgent00.obj
 0003:00000050       AGENT_FINISHED_METHOD_SIGNATURE 0000000180009050     libattach002aAgent00.obj
 0003:00000058       testEvents                 0000000180009058     libattach002aAgent00.obj
 0003:0001aba0       nsk_context                0000000180023ba0     libattach002aAgent00.obj
 0003:0001abac       redefineAttempted          0000000180023bac     libattach002aAgent00.obj
 0003:0001abb0       redefineSucceed            0000000180023bb0     libattach002aAgent00.obj
 0003:0001abb4       agentFailed                0000000180023bb4     libattach002aAgent00.obj
 0003:0001abb8       agentThread                0000000180023bb8     libattach002aAgent00.obj
 0003:0001abc0       context                    0000000180023bc0     libattach002aAgent00.obj
 0003:0001ac78       agentThreadProc            0000000180023c78     libattach002aAgent00.obj
 0003:0001ac80       agentThreadArg             0000000180023c80     libattach002aAgent00.obj
 0003:0001ac88       agent_data                 0000000180023c88     libattach002aAgent00.obj
 0003:0001ac98       jvmti_env                  0000000180023c98     libattach002aAgent00.obj
 0003:0001aca0       jvm                        0000000180023ca0     libattach002aAgent00.obj
 0003:0001aca8       jni_env                    0000000180023ca8     libattach002aAgent00.obj
 0003:0001acb0       currentAgentStatus         0000000180023cb0     libattach002aAgent00.obj
 0003:0001acb4       ?codeAttributeIndex@@3GA   0000000180023cb4     libattach002aAgent00.obj
 0003:0001acb8       checkStatus_func           0000000180023cb8     libattach002aAgent00.obj
 0003:0001acc0       ?lineNumberAttributeIndex@@3GA 0000000180023cc0     libattach002aAgent00.obj
 0003:0001acc4       ?localVarAttributeIndex@@3GA 0000000180023cc4     libattach002aAgent00.obj
 0003:0001acc8       ?localVarTypeAttributeIndex@@3GA 0000000180023cc8     libattach002aAgent00.obj
 0003:0001accc       ?stackMapAttributeIndex@@3GA 0000000180023ccc     libattach002aAgent00.obj
 0003:0001acd0       ?stackFrameOffset@@3GA     0000000180023cd0     libattach002aAgent00.obj
 0003:0001acd4       ?mode@@3HA                 0000000180023cd4     libattach002aAgent00.obj
 0003:0001acd8       ?orig@@3PEBEEB             0000000180023cd8     libattach002aAgent00.obj
 0003:0001ace0       ?gen@@3PEAEEA              0000000180023ce0     libattach002aAgent00.obj
 0003:0001ace8       ?inputPos@@3PEAEEA         0000000180023ce8     libattach002aAgent00.obj
 0003:0001acf0       ?endPos@@3PEBEEB           0000000180023cf0     libattach002aAgent00.obj
 0003:0001acf8       ?genPos@@3PEAEEA           0000000180023cf8     libattach002aAgent00.obj
 0003:0001ad00       ?markPos@@3PEAEEA          0000000180023d00     libattach002aAgent00.obj
 0003:0001ad08       ?constantPool@@3PEAPEADEA  0000000180023d08     libattach002aAgent00.obj
 0003:0001ad10       ?constantPoolSize@@3GA     0000000180023d10     libattach002aAgent00.obj
 0003:0001ad14       ?constantPoolCount@@3GA    0000000180023d14     libattach002aAgent00.obj
 0003:0001ad18       ?zeroBytes@@3PAEA          0000000180023d18     libattach002aAgent00.obj
 0003:0001ad1c       ?codeLength@@3IA           0000000180023d1c     libattach002aAgent00.obj
 0003:0001ad20       ?map@@3PEAIEA              0000000180023d20     libattach002aAgent00.obj
 0003:0001ad28       ?widening@@3PEACEA         0000000180023d28     libattach002aAgent00.obj
 0003:0001ad30       internalError              0000000180023d30     libattach002aAgent00.obj
 0003:0001ad34       multiagentsCount           0000000180023d34     libattach002aAgent00.obj
 0003:0001ad38       targetAppClass             0000000180023d38     libattach002aAgent00.obj
 0003:0001ad40       agentLoadedMethod          0000000180023d40     libattach002aAgent00.obj
 0003:0001ad48       agentFinishedMethod        0000000180023d48     libattach002aAgent00.obj
 0003:0001ad50       options                    0000000180023d50     libattach002aAgent00.obj
 0003:0001ad58       agentName                  0000000180023d58     libattach002aAgent00.obj
 0003:0001ad70       GS_ExceptionRecord         0000000180023d70     MSVCRT:gs_report.obj
 0003:0001ae10       GS_ContextRecord           0000000180023e10     MSVCRT:gs_report.obj
 0003:0001b2e0       ?g_tss_cv@@3U_RTL_CONDITION_VARIABLE@@A 00000001800242e0     MSVCRT:thread_safe_statics.obj
 0003:0001b2e8       ?g_tss_event@@3PEAXEA      00000001800242e8     MSVCRT:thread_safe_statics.obj
 0003:0001b2f0       ?g_tss_mutex@@3U_RTL_CRITICAL_SECTION@@A 00000001800242f0     MSVCRT:thread_safe_statics.obj
 0003:0001b318       ?g_sleep_condition_variable_cs@@3P6AHPEAU_RTL_CONDITION_VARIABLE@@PEAU_RTL_CRITICAL_SECTION@@K@ZEA 0000000180024318     MSVCRT:thread_safe_statics.obj
 0003:0001b320       ?g_wake_all_condition_variable@@3P6AXPEAU_RTL_CONDITION_VARIABLE@@@ZEA 0000000180024320     MSVCRT:thread_safe_statics.obj
 0003:0001b32c       ?__proc_attached@@3HA      000000018002432c     MSVCRT:dll_dllmain.obj
 0003:0001b340       ?is_initialized_as_dll@@3_NA 0000000180024340     MSVCRT:utility.obj
 0003:0001b341       ?module_local_atexit_table_initialized@@3_NA 0000000180024341     MSVCRT:utility.obj
 0003:0001b348       ?module_local_atexit_table@@3U_onexit_table_t@@A 0000000180024348     MSVCRT:utility.obj
 0003:0001b360       ?module_local_at_quick_exit_table@@3U_onexit_table_t@@A 0000000180024360     MSVCRT:utility.obj
